:020000040800F2
:1000000000060020E1020008E3020008E302000805
:10001000E3020008E3020008E3020008E30200082C
:10002000E3020008E3020008E30200085970000838
:10003000E3020008E3020008E3020008E30200080C
:10004000E3020008E3020008E3020008E3020008FC
:10005000E3020008E3020008E3020008E3020008EC
:10006000E3020008E3020008E30200081D4600085E
:1000700045460008714600089D460008C94600082C
:10008000F14600081D470008E3020008E3020008EB
:10009000E3020008E3020008E3020008E3020008AC
:1000A000E3020008E3020008E3020008E30200089C
:1000B000797F0008E3020008E3020008E302000879
:1000C000E3020008E3020008E3020008E30200087C
:1000D000E3020008E3020008E3020008E30200086C
:1000E000E3020008E3020008E3020008E30200085C
:1000F000E3020008E3020008E302000849470008A1
:10010000E3020008657F0008E3020008E30200083C
:10011000E3020008E3020008E3020008E30200082B
:10012000754700089D470008C9470008F5470008C3
:1001300021480008E3020008E3020008E302000887
:10014000E3020008E3020008E3020008E3020008FB
:100150004948000875480008A1480008E302000863
:10016000E3020008E3020008E3020008E3020008DB
:10017000E3020008457C0008E3020008E3020008EF
:10018000E3020008E3020008E3020008E3020008BB
:10019000E3020008E3020008E3020008E3020008AB
:1001A000E3020008E3020008E3020008E30200089B
:1001B000E3020008E3020008E3020008E30200088B
:1001C000E3020008E3020008E3020008E30200087B
:1001D000E3020008317C0008E3020008E3020008A3
:1001E000E3020008E3020008E3020008E30200085B
:1001F000E3020008E3020008E3020008E30200084B
:10020000E3020008E3020008E3020008E30200083A
:10021000E3020008E3020008E3020008E30200082A
:10022000E3020008E3020008E3020008E30200081A
:10023000E3020008E3020008E3020008E30200080A
:10024000E3020008E3020008E3020008E3020008FA
:10025000E3020008E3020008E3020008E3020008EA
:10026000E3020008E3020008E3020008E3020008DA
:10027000E3020008E3020008E3020008E3020008CA
:10028000E3020008E3020008E3020008E3020008BA
:10029000E3020008E3020008E3020008E3020008AA
:1002A000E3020008E3020008E3020008E30200089A
:1002B000E3020008E3020008E3020008E30200088A
:1002C000E3020008E3020008E3020008E30200087A
:1002D000E3020008E3020008E3020008E30200086A
:1002E00002E000F000F8FEE772B6374880F30888B5
:1002F000364880F3098836483649086040F20000E5
:10030000CCF200004EF63471CEF200010860BFF36B
:100310004F8FBFF36F8F40F20000C0F2F0004EF637
:100320008851CEF200010860BFF34F8FBFF36F8F8B
:100330004FF00000E1EE100A4EF63C71CEF20001E3
:100340000860062080F31488BFF36F8F06F0E6FE86
:1003500006F06CF84FF055301F491B4A91423CBFE4
:1003600041F8040BFAE71D49184A91423CBF41F895
:10037000040BFAE71A491B4A1B4B9A423EBF51F83D
:10038000040B42F8040BF8E700201849184A914280
:100390003CBF41F8040BFAE706F0FEFE06F0CAF88F
:1003A000144C154DAC4203DA54F8041B8847F9E7A6
:1003B00000F0C4F9114C124DAC4203DA54F8041B9E
:1003C0008847F9E706F0E6BE00060020002200207C
:1003D0000000000808ED00E00000002000060020FA
:1003E0008093000800220020642200206822002060
:1003F00044590020E0020008E0020008E002000882
:10040000E00200082DE9F04F2DED108AC1F80CD064
:10041000D0F80CD0BDEC108ABDE8F08F002383F338
:1004200011882846A047002005F0E2FDFEE705F010
:100430003BFD00DFFEE7000053B94AB9002908BFC1
:1004400000281CBF4FF0FF314FF0FF3000F074B9AF
:10045000ADF1080C6DE904CE00F006F8DDF804E01B
:10046000DDE9022304B070472DE9F047089D0446FA
:100470008E46002B4DD18A42944669D9B2FA82F257
:1004800052B101FA02F3C2F1200120FA01F10CFA93
:1004900002FC41EA030E94404FEA1C48210CBEFBCB
:1004A000F8F61FFA8CF708FB16E341EA034306FB54
:1004B00007F199420AD91CEB030306F1FF3080F0E3
:1004C0001F81994240F21C81023E63445B1AA4B230
:1004D000B3FBF8F008FB103344EA034400FB07F7D2
:1004E000A7420AD91CEB040400F1FF3380F00A8113
:1004F000A74240F207816444023840EA0640E41B08
:1005000000261DB1D4400023C5E900433146BDE8B3
:10051000F0878B4209D9002D00F0EF800026C5E955
:10052000000130463146BDE8F087B3FA83F6002E6D
:100530004AD18B4202D3824200F2F980841A61EBE5
:10054000030301209E46002DE0D0C5E9004EDDE703
:1005500002B9FFDEB2FA82F2002A40F09280A1EBEB
:100560000C014FEA1C471FFA8CFE0126200CB1FB40
:10057000F7F307FB131140EA01410EFB03F0884239
:1005800008D91CEB010103F1FF3802D2884200F2C6
:10059000CB804346091AA4B2B1FBF7F007FB101158
:1005A00044EA01440EFB00FEA64508D91CEB0404F6
:1005B00000F1FF3102D2A64500F2BB800846A4EB51
:1005C0000E0440EA03409CE7C6F12007B34022FA3C
:1005D00007FC4CEA030C20FA07F401FA06F31C436B
:1005E000F9404FEA1C4900FA06F3B1FBF9F8200C78
:1005F0001FFA8CFE09FB181140EA014108FB0EF0BE
:10060000884202FA06F20BD91CEB010108F1FF3A0D
:1006100080F08880884240F28580A8F10208614419
:10062000091AA4B2B1FBF9F009FB101144EA014127
:1006300000FB0EFE8E4508D91CEB010100F1FF34D2
:100640006CD28E456AD90238614440EA0840A0FB6A
:100650000294A1EB0E01A142C846A64656D353D040
:100660005DB1B3EB080261EB0E0101FA07F722FA64
:1006700006F3F1401F43C5E9007100263146BDE88D
:10068000F087C2F12003D8400CFA02FC21FA03F3F0
:10069000914001434FEA1C471FFA8CFEB3FBF7F071
:1006A00007FB10360B0C43EA064300FB0EF69E4296
:1006B00004FA02F408D91CEB030300F1FF382FD22F
:1006C0009E422DD9023863449B1B89B2B3FBF7F6D7
:1006D00007FB163341EA034106FB0EF38B4208D9B0
:1006E0001CEB010106F1FF3816D28B4214D9023EF1
:1006F0006144C91A46EA004638E72E46284605E70F
:100700000646E3E61846F8E64B45A9D2B9EB0208DF
:1007100064EB0C0E0138A3E74646EAE7204694E76F
:100720004046D1E7D0467BE7023B614432E73046A2
:1007300009E76444023842E7704700BF38B501F06A
:100740007FFA01F007FC06F091FB054606F07AFC03
:100750000446D0B90F4B9D4219D001339D4241F25E
:10076000883504BF01240025002006F089FB0CB168
:1007700000F076F801F0C2FB00F02EFD08B100F0A9
:100780006FF8284600F01AF9F9E70025ECE705466E
:10079000EAE700BF010007B008B501F023FAA0F1B5
:1007A00020035842584108BD07B5042101900DEBC4
:1007B000010001F035FA03B05DF804FB38B53023D1
:1007C00083F31188174803680BB105F0F5FC00238B
:1007D000154A4FF47A71134805F0E4FC002383F3C3
:1007E0001188124C236813B12368013B23606368AE
:1007F00013B16368013B63600D4D2B7833B96368B7
:100800007BB9022001F0E4FA322363602B78032BDA
:1008100007D163682BB9022001F0DAFA4FF47A733A
:10082000636038BD68220020BD07000888230020CF
:1008300080220020084B187003280CD8DFE800F055
:1008400008050208022001F0B9BA022001F0ACBA92
:10085000024B00225A60704780220020882300202B
:10086000F8B5504B504A1C461968013100F0998088
:1008700004339342F8D162684C4B9A4240F2918023
:100880004B4B9B6803F1006303F500339A4280F001
:100890008880002001F0FAF90220FFF7CBFF454BDA
:1008A0000021D3F8E820C3F8E810D3F81021C3F8EA
:1008B0001011D3F81021D3F8EC20C3F8EC10D3F8C2
:1008C0001421C3F81411D3F81421D3F8F020C3F87D
:1008D000F010D3F81821C3F81811D3F81821D3F861
:1008E000802042F00062C3F88020D3F8802022F0FC
:1008F0000062C3F88020D3F88020D3F8802042F033
:100900000072C3F88020D3F8802022F00072C3F870
:100910008020D3F8803072B64FF0E023C3F8084D42
:10092000D4E90004BFF34F8FBFF36F8F224AC2F8A0
:100930008410BFF34F8F536923F480335361BFF3A7
:100940004F8FD2F8803043F6E076C3F3C905C3F386
:100950004E335B0103EA060C29464CEA81770139E4
:10096000C2F87472F9D2203B13F1200FF2D1BFF319
:100970004F8FBFF36F8FBFF34F8FBFF36F8F5369ED
:1009800023F4003353610023C2F85032BFF34F8F7A
:10099000BFF36F8F302383F31188854680F3088877
:1009A0002047F8BD0000020820000208FFFF0108F0
:1009B000002200200044025800ED00E02DE9F04F35
:1009C00095B0DFF8D8922022FF21029004A8D9F830
:1009D000085001F03DFAA84A1378A3B90121A748AD
:1009E00011700360302383F3118803680BB105F0A5
:1009F000E3FB0023A24A4FF47A71A04805F0D2FB32
:100A0000002383F31188029B13B19E4B029A1A6054
:100A10009D4A1378032B03D000231370994A536027
:100A20004FF0000B029C5E46DA46CDF804B0012080
:100A300001F0C4F924B1934B1B68002B00F028820D
:100A4000002001F0CFF8B0F10008F3DB012001F045
:100A5000ABF9A8F121031F2BE9D801A252F823F02A
:100A6000E10A0008FD0A00088B0B00082F0A0008A5
:100A70002F0A00082F0A0008150C0008070E0008AE
:100A8000F90C0008550D00087B0D0008A10D0008A9
:100A90002F0A0008B30D0008D70D00084F0E0008FC
:100AA000690B00082F0A0008970E0008ED0A0008DD
:100AB000690B00082F0A0008550D00082F0A0008CE
:100AC0002F0A00082F0A00082F0A00082F0A000822
:100AD0002F0A00082F0A00082F0A00088B0B0008B5
:100AE0000220FFF759FE002840F0FF81029B0221FF
:100AF0006648BBF1000F08BF1C4640E04FF47A7017
:100B000001F070F8071EF1DB0220FFF745FE002818
:100B1000ECD0013F052F00F2EA81DFE807F0030780
:100B20000A0D10330520FFF73FFE14E0D9F800004E
:100B3000F9E7D9F80400F6E7D9F80800F3E74FF031
:100B40001C08404608F1040801F0A2F8FFF72CFE4B
:100B5000B8F12C0FF5D10120019B4FF0000A00FAEB
:100B600007F71F43FBB2019301F0BEF92EB1019BC1
:100B700003F00B030B2B08BF00240221444801F0B3
:100B80004FF854E7D9F80C00CDE7002EAED0019B0A
:100B900003F00B030B2BA9D10220FFF7FDFD074645
:100BA0000028A3D00120002601F070F80220FFF7F2
:100BB00041FE1FFA86FB584601F078F8044688B1DA
:100BC000A8F14002584601365142514101F07EF8E9
:100BD0000028EED1BB46044602212E483E4601F0D5
:100BE0001FF824E725460120FFF724FED9F8083036
:100BF000AB4207D9284601F04BF8013040F07A812A
:100C00000435F3E70025204BBB463E461D701D4BC7
:100C10005D60A9E7002E3FF469AF019B03F00B0371
:100C20000B2B7FF463AF0220FFF704FE322000F0AD
:100C3000D9FFB0F10008FFF659AF18F003077FF4B1
:100C400055AF08EB0503D9F8082093423FF64EAFA5
:100C5000B8F5807F3FF74AAF0F4BB84503931FDDD0
:100C60004FF47A7000F0BEFF0028FFF63FAF039B01
:100C7000013703F8010BF0E78423002068220020ED
:100C8000BD07000888230020802200206C8900080E
:100C9000648900086889000884220020002200205E
:100CA000C820FFF779FD074600283FF41FAF1F2D2E
:100CB00011D8C5F1200204AB25F003008F4942454D
:100CC000184428BF4246039201F09CF8039AFF2182
:100CD0008A4801F0BDF84FEAA803C8F387028749A4
:100CE0002846039301F0BCF8064600283FF474AF91
:100CF000039B05EB830537E70220FFF74DFD002836
:100D00003FF4F4AE01F000F800283FF4EFAE002706
:100D1000B846D9F80830BB4218D91F2F11D8049B08
:100D200001330ED027F0030314AA134453F8403CB8
:100D30000C93404604220CA9043701F01DF98046AB
:100D4000E7E7384600F0A4FF0C90F2E74046FFF7D3
:100D50002BFD09E7002364210CA80C9300F056FF3B
:100D600000287FF4C3AE0220FFF716FD00283FF4F1
:100D7000BDAE0C9800F0BEFFE9E7002364210CA88B
:100D80000C9300F043FF00287FF4B0AE0220FFF781
:100D900003FD00283FF4AAAE0C9800F0ADFFD6E7A3
:100DA0000220FFF7F9FC00283FF4A0AE00F0BCFFE2
:100DB000CDE70220FFF7F0FC00283FF497AE0CA926
:100DC000142000F0B7FF0390FFF7EEFC03990CA886
:100DD00000F026FFC8E60220FFF7DEFC00283FF403
:100DE00085AE474B0CAF03F1100C1868083353F86D
:100DF000041C3A46634503C21746F6D11020FFF79C
:100E0000D3FC1021E3E7322000F0ECFE071EFFF6D2
:100E10006DAEBB077FF46AAE07EB0A03D9F8082072
:100E200093423FF663AE0220FFF7B6FC00283FF482
:100E30005DAE27F003075744BA453FF495AE5046E0
:100E40000AF1040A00F024FFFFF7AEFCF4E74FF4C8
:100E50007A70FFF7A1FC00283FF448AE00F054FF81
:100E6000002849D0049B01330BD0082204A900209C
:100E700000F0F6FF00283FD02022FF2104A800F058
:100E8000E7FF2048022100F0CBFE1F4805F0B6F82E
:100E900015B0BDE8F08F002E3FF428AE019B03F0A3
:100EA0000B030B2B7FF422AE002364210CA80C93C0
:100EB00000F0ACFE074600287FF418AE0220FFF7D2
:100EC0006BFC804600283FF411AE02210D4800F073
:100ED000A7FE41F2883005F091F80C9801F038F83F
:100EE00046463C4601F000F8A1E506463CE64FF0D8
:100EF000000AFBE5BB466FE637466DE6842200201C
:100F00005089000864890008A0860100704700002D
:100F100070470000704700002DE9F04100F5803770
:100F2000044616463B7C5BB9C0681030204400F094
:100F300069FFE5683544B5F5004FE56002D816B1A4
:100F4000BDE8F081DEB905F07F0605F11000002153
:100F5000C6F180062044F6B232462E4400F078FFF7
:100F6000A06804F11008324600F10060414600F527
:100F7000003005F01BFD30B901233B74E0E74FF46E
:100F800000463546ECE7A26805F1100140463244C0
:100F90002144A260E268521BE26000F033FF0220AD
:100FA000BDE8F04100F014BF183000F0E9BC0000CB
:100FB00010B5044600F0FCFF204610BD10B50446F5
:100FC00000F0F6FF204610BDC0B2A0F14103052B92
:100FD00002D83738C0B27047A0F16103052B94BF27
:100FE00057383038F6E7000070B504461546084615
:100FF00003220C4900F010FF014688B908346E1C2A
:1010000015F91100FFF7E0FF024616F91100013152
:10101000FFF7DAFF102940EA021004F8010BEFD1C4
:1010200070BD00BF708900082DE9F04FADF53F7D20
:101030000746416801222AA802F09CFE002840F0E1
:1010400087800646824681461125DFF80C81DFF84D
:101050000CB101AB4FF4805241462AA802F0EAFFDE
:10106000002875D1019AB2F5805F71D8002A65D049
:101070000446019A9442ECD2282D0FD008DC132D9F
:101080002DD01E2D39D0112D13D00134A4B2F0E78C
:10109000322D2DD0372D2FD02D2DF6D13B68121BA0
:1010A00008EB040138461B692D259847BDF804401C
:1010B000EBE7121B022A09D9594608EB040000F09D
:1010C000ABFE18B902342825A4B2DEE718F80430C4
:1010D0003A2B3DD00A2B1CBFA1461325D5E718F8A3
:1010E00004300A2B34D03A2B04BFA2463225CCE779
:1010F00018F80430202BC8D0264618F804300A2BE4
:101100001AD1AAEB090208EB090102A811254F2AFE
:1011100028BF4F2207F008FCA21B08EB060116A807
:101120004F2A28BF4F2207F0FFFB3B6816AA02A9EF
:10113000DB6838469847A8E71E25A6E73B6838468F
:1011400004491B69984701200DF53F7DBDE8F08FEC
:101150000020F9E7728A00089023002074890008B3
:1011600000F1180110B5044686B00846019100F060
:10117000F1FB2046FFF758FF60B1019902A800F08B
:1011800049FC102204F1080102A807F08DFBB0FA17
:1011900080F0400906B010BD70B504460025EEB2DF
:1011A000304600F083FD58B100213046013500F093
:1011B0008DFD08B9002070BD022000F009FEEEE7A9
:1011C0002046FFF731FF0028F4D004F58034207C5E
:1011D00080F00100EFE70000F0B5C9B005F05EFE59
:1011E00000F002FF18B90025284649B0F0BD694655
:1011F0002A4802F0E1FF00284BD1294C204603F099
:101200000BF8284803F008F8274803F005F82146B2
:10121000224803F07DF80028E5D1702000F0C2FEDE
:10122000064610B1214B44600360336830469B682A
:101230009847054600282ED01A4F1948394603F022
:1012400067F805460028CED1194800F0ABFE0446E9
:1012500038B1184B4760036000F58033C0E9025590
:101260001D74236820469B689847054628B10E499F
:101270000C4803F04DF80028B5D1336830465B6860
:1012800098471CB1236820465B68984700F094FE9D
:10129000AAE70025FAE70446EFE700BF78890008CF
:1012A000888900089F890008B5890008D889000846
:1012B00014000100F48900082DE9F04FD44A8DB0E4
:1012C0000B68D0F804A001931A440368D14E1A4465
:1012D000D1F81C90DFF8B4C3DFF8B4B3D0E902341E
:1012E000634003EA0A03634013444A6802920AEB2C
:1012F0007363029CC84A2244C468224484688AEA10
:1013000004051D40654015448A68039203EB35557A
:10131000039CC24A2244846822448AEA03042C4083
:1013200084EA0A041444CA6805EBF43404921644AF
:1013300083EA0502224056445A4032440E6905961B
:1013400004EBB222059FB64E3E441E4485EA0403D8
:1013500013406B4033444E69069602EB7363069F5D
:10136000B04E3E442E4484EA02051D40654035449B
:101370008E69079603EB3555079FAB4E3E442644D6
:1013800082EA03042C4054403444A84E4E4405EBFA
:10139000F434164483EA050222405A4032440E6A6D
:1013A000089604EBB222089FA14E3E441E4485EAF3
:1013B000040313406B4033444E6A099602EB736397
:1013C000099F9C4ED1F830E03E44D1F83880F34478
:1013D0002E4484EA02051D40654035448E6AA6F518
:1013E000244703EB35550A964F3F274482EA03040E
:1013F0002C4054403C44CF6A0B9705EBF4340B9ED1
:101400008D4F3744029E174483EA050222405A401A
:101410003A448A4F774404EBB2221F4485EA04031E
:1014200013406B403B444F6BBC4402EB7363654419
:1014300084EA020C0CEA030C8CEA040C6544DFF825
:1014400054C2C44403EB3555A44482EA03042C403F
:1014500054406444D1F83CC0794905EBF43461440C
:10146000114483EA050222405A400A44754904EBBC
:10147000B2223144079E194484EA02032B406340A0
:101480000B44714902EBF36331440B9E0D4482EA35
:1014900003012140514029446C4D03EBF151354487
:1014A000019E254483EA010414405C402C44684DAD
:1014B00001EBB4443544069E154481EA04021A4007
:1014C0004A402A44634D04EB323235440A9E1D449F
:1014D00084EA02030B4063402B445F4D02EBF3634D
:1014E0003544059E0D4482EA0301214051402944C0
:1014F0005A4D03EBF1516544254483EA010414403D
:101500005C402C44564D01EBB4443544099E1544CF
:1015100081EA04021A404A402A44524D04EB323216
:101520003544049E1D4484EA02030B4063402B446F
:101530004D4D02EBF36345440D4482EA0301214023
:1015400051402944494D03EBF1513544089E2C4448
:1015500083EA010515405D402C44454D01EBB44440
:101560003544039E2A4481EA04051D404D402A4427
:10157000404D04EB32323D442B4484EA020593444F
:101580000D4065402B443C4D02EBF3633544069E11
:10159000294482EA0305254055402944374D03EB91
:1015A000F1514D442C4483EA010515405D4025442A
:1015B00001EBB54581EA050404EA03024A405A44B6
:1015C000A6F5B82B089E05EB3232ABF2BE6B544049
:1015D0005B4423442A4C344402EB33730B9E0C448B
:1015E00085EA020159402144264C344403EB7151F1
:1015F000029E254482EA03044C402544224C444484
:1016000001EB3545144483EA01026A40224443E079
:1016100078A46AD7EECEBDC156B7C7E8DB702024E8
:10162000AF0F7CF52AC68747134630A8019546FDC3
:10163000D8988069AFF7448BBED75C892211906B34
:101640002108B44962251EF640B340C0515A5E26B7
:10165000AAC7B6E95D102FD65314440281E6A1D87B
:10166000C8FBD3E7E6CDE121D60737C3870DD5F414
:10167000ED145A4505E9E3A9F8A3EFFCD9026F6719
:1016800081F6718722619D6D0C38E5FD937198FD9F
:101690008A4C2A8D8E4379A6934C344405EB7222F2
:1016A000059E1C4481EA0503534023448F4C344477
:1016B00002EB33730A9E0C4485EA0201594021442F
:1016C0008B4C4C4403EB7151254482EA03044C409B
:1016D0002C44884D354401EB3444019E154483EA83
:1016E000010262402A44844D3D4404EB72221D44B1
:1016F00081EA040353402B44804D354402EB33739D
:10170000049E294484EA02055D4029447C4D354409
:1017100003EB7151079E254482EA03044C402C449C
:10172000784D354401EB3444099E2A4483EA01058F
:1017300065401544744A324404EB7525039E1344F6
:1017400081EA04026A401A44704B734405EB32721A
:101750000B4484EA0501514019446D4B634402EB8C
:1017600071511C4485EA02034B401C44694B3344CD
:1017700001EB3444019E1D4482EA010363402B4483
:10178000654D04EB73233544069E154463EA01025C
:1017900062402A44614D03EBB2624D4462EA04099F
:1017A00029445F4D89EA0309454449442C445D4D71
:1017B00002EBB1513544049E61EA03081D4488EAF6
:1017C0000208444401EB744464EA02034B402B4496
:1017D000554D04EBF323754463EA010E15448EEA7C
:1017E000040E0EEB0502514D03EBB262354462EA82
:1017F000040E29440A9D8EEA030EA5F580164C4D71
:101800007144A6F6833602EBB151264461EA030423
:1018100054403444029E01EB7444354464EA0206A9
:101820001D444E407319089E424D04EBF32335448A
:1018300063EA01061544664072193F4D03EBB2623C
:10184000654462EA040629443C4D5E403144079EEB
:1018500002EBB151354461EA03062C44384D564041
:101860003D443444059E1D4401EB744464EA020384
:101870004B402B44334D04EBF32335440B9E15446E
:1018800063EA010262402A442F4D03EBB262354401
:10189000039E0D4462EA0401594029442B4D02EB9A
:1018A000B15135442A4E254461EA030454402C4486
:1018B000099D01EB74442E4464EA02051E4485EA46
:1018C00001039D1903681A440AEB040303EBF52393
:1018D0000260436083681C44C36819448460C1602B
:1018E0000DB0BDE8F08F00BF44EABEA4A9CFDE4B27
:1018F000604BBBF670BCBFBEC67E9B28FA27A1EA30
:101900008530EFD4051D880439D0D4D9E599DBE6BC
:10191000F87CA21F6556ACC4442229F497FF2A43E1
:10192000A72394AB39A093FCC3595B6592CC0C8F71
:10193000D15D84854F7EA86FE0E62CFE144301A3A1
:10194000A111084E827E53F735F23ABDBBD2D72A99
:1019500091D386EB094B036003F18833436003F1B5
:101960002943A3F59613A3F68B638360A3F1883311
:10197000C3600023C0E90433704700BF01234567FB
:101980002DE9F8431446026905460E46E300C2F30A
:10199000C50800F118079B18036122BF4369013392
:1019A000436112F4FC7F436903EB5473436114D029
:1019B000C8F1400907EB08004C4504D22246BDE8B7
:1019C000F84306F081BF403C4A464E4406F07CFF97
:1019D000444439462846FFF76FFCA04606EB04094D
:1019E000B8F13F0FA9EB08010AD94022384606F0AA
:1019F0006BFF39462846A8F14008FFF75DFCEFE78A
:101A0000A1096FF03F02384602FB014206EB81114B
:101A1000D5E7000070B50B6901F1180506460C46C4
:101A2000C3F3C503EA18501C8022EA54C3F13F02F5
:101A3000072A1FD8002100F00BFA29462046FFF79D
:101A40003BFC38220021284600F002FA236929468F
:101A50002046236563696365FFF72EFC214610224B
:101A6000304606F031FF204658220021BDE8704084
:101A700000F0EEB9C3F137020021E5E70F4B70B576
:101A80001B780C460133DBB2012B11D80C4D4FF4FF
:101A90007A732968A2FB033222460E6A0146284661
:101AA000B047844204D1074B002201201A7070BD58
:101AB0004FF4FA7004F0A2FA0020F8E71022002098
:101AC000A83B0020BC33002000232DE9F0471A4634
:101AD000054688460120194602F08AFF0446802008
:101AE00005F082F80746002861D0002C5FD03B4EFD
:101AF00028464FF0800A736943F0C0637361D6F8DB
:101B0000143143F0C063C6F8143104F0EFFE05EB66
:101B1000080200FB05F34FF4D06C50434FF03D0E2C
:101B2000834233D23269520143D4D6F81021510195
:101B30003FD4216803F100628A602268D76022687E
:101B4000C2F804A02268C2F800C0D4F80090D9F806
:101B5000002042F00102C9F80020D4F80090D9F822
:101B6000002022F01E02C9F80020D4F80090D9F815
:101B70000020D207FBD494F80C90803361680EFAF1
:101B800009F20A60CCE7002004F08EFF204602F044
:101B90006FFF384605F064F8104B5A6942F0C06296
:101BA0005A61D3F8142142F0C062C3F81421BDE891
:101BB000F0870B4B9A6A42F400729A629A6A42F476
:101BC00000429A6261B60026012004F06DFFB04524
:101BD000D9D9A819013604F0A1FEF8E70020005277
:101BE00000ED00E0002307B5024601210DF10700DA
:101BF0008DF80730FFF742FF20B19DF8070003B0D2
:101C00005DF804FB4FF0FF30F9E700000A460421BD
:101C100008B5FFF733FF80F00100C0B2404208BDB5
:101C200030B4054C0A46014623682046DD69034B63
:101C3000AC4630BC604700BFA83B0020A086010036
:101C400070B5104C0025104E04F054FE2080306812
:101C5000238883420CD800252088013804F046FEF2
:101C600023880544013BB5F5802F2380F4D370BD54
:101C700004F03CFE336805440133B5F5003F3360A2
:101C8000E5D3E8E7BE3300209033002004F00CBF1A
:101C900000F1006000F500300068704700F100605E
:101CA000920000F5003004F081BE0000054B1A6878
:101CB000054B1B889B1A834202D9104404F016BEC0
:101CC0000020704790330020BE33002038B5044612
:101CD000074D29B128682044BDE8384004F01EBEF5
:101CE0002868204404F008FE0028F3D038BD00BF67
:101CF000903300200020704700F1FF5000F58F1056
:101D0000D0F8000870470000064991F8243033B13C
:101D100000230822086A81F82430FFF7BFBF0120A2
:101D2000704700BF94330020014B1868704700BF14
:101D30000010005C194B01380322084470B51D687F
:101D4000174BC5F30B042D0C1E88A6420BD15C6803
:101D50000A46013C824213460FD214F9016F4EB17C
:101D600002F8016BF6E7013A03F10803ECD1814276
:101D70000B4602D22C2203F8012B0424094A1688B0
:101D8000AE4204D1984284BF967803F8016B013CBF
:101D900002F10402F3D1581A70BD00BF0010005CBC
:101DA00014220020348A0008022803D1024B4FF489
:101DB00000429A61704700BF00040258022803D114
:101DC000024B4FF000429A61704700BF0004025876
:101DD000022804D1024A536983F4004353617047D7
:101DE0000004025870B504464FF47A764CB1412C89
:101DF000254628BF412506FB05F0641B04F0FEF8CC
:101E0000F4E770BD002310B5934203D0CC5CC454FA
:101E10000133F9E710BD0000013810B510F9013F9A
:101E20003BB191F900409C4203D11AB10131013A12
:101E3000F4E71AB191F90020981A10BD1046FCE79A
:101E400003460246D01A12F9011B0029FAD1704745
:101E500002440346934202D003F8011BFAE770479D
:101E60002DE9F8431F4D14460746884695F824206F
:101E700052BBDFF870909CB395F824302BB9202228
:101E8000FF2148462F62FFF7E3FF95F82400414603
:101E9000C0F1080205EB8000A24228BF2246D6B25C
:101EA0009200FFF7AFFF95F82430A41B17441E449F
:101EB0009044E4B2F6B2082E85F82460DBD1FFF737
:101EC00023FF0028D7D108E02B6A03EB820383426B
:101ED000CFD0FFF719FF0028CBD10020BDE8F88351
:101EE0000120FBE794330020024B1A78024B1A7052
:101EF000704700BFBC3300201022002010B5114CE9
:101F0000114803F083FB21460F4803F0ABFB246824
:101F10004FF47A70D4F89020D2F8043843F00203DA
:101F2000C2F80438FFF75EFF0849204603F0A8FC1A
:101F3000D4F89020D2F8043823F00203C2F8043811
:101F400010BD00BFF0910008A83B0020F8910008E8
:101F50007047000008B571B6054B1988054B188805
:101F6000FFF7B2FD02210E20FFF7AEFD61B608BDFE
:101F7000BE3300209033002030B50A44084D914212
:101F80000DD011F8013B5840082340F30004013BF9
:101F90002C4013F0FF0384EA5000F6D1EFE730BD88
:101FA0002083B8ED0121884238BF084604F054BEB2
:101FB00008B104F055BE704710B5084C012208491D
:101FC000002001F0B3FE23783BB1064803F05EFA2F
:101FD000044803F091FA0023237010BDC0330020A1
:101FE000448A0008A03600201D482DE9F041036D09
:101FF0002BB901224FF48051503004F075FF194E77
:1020000033780BB1FFF7D8FF0324174F4FF00008C8
:10201000134D15492846C7F8048003F05FFA284697
:1020200003F098F848B1013C284603F065FA14F033
:10203000FF04EED1204634700FE00C4901220C4819
:1020400001F074FE014618B1284603F01FFAEAE7D2
:10205000084800F011F801203070BDE8F08100BFA1
:10206000A0360020C03300202C220020448A000823
:10207000C4330020488A00080FB4002004B0704721
:102080000068704703460068596870470B0A017082
:1020900043700B0C090E8370C1707047110A0270F7
:1020A00003714170110C120E8170C2701A0A4271D4
:1020B0001A0C1B0E8271C37170470000C36A02398B
:1020C000023B8B4283BF4389006C01FB030000206D
:1020D00070470000C2F307238A76CB760378032B80
:1020E00001BF120C0A75120A4A75704700F10B0104
:1020F0000022D30143EA520310F8012B52FA83F372
:102100008842DAB2F5D110467047000010B5417828
:1021100004460020013102464901022A16BFA35C91
:10212000032203EBC03302F101021EBF9BB203EB9B
:10213000500398B29142F0D810BD000002684AB135
:10214000134613F8011B1F290DD93A29F9D1911C07
:102150008B4202D04FF0FF3070471278302AF9D10D
:10216000036000207047014B18787047103600203C
:1021700038B50D46044618B9092000232B6038BD38
:102180000368002BF8D01A78002AF5D08188DA8805
:102190009142F1D1587804F0CDF810F00100EBD164
:1021A0002368EBE738B50D4640F25231144602F091
:1021B000B9F9FF2807D9012C0BD9030A022468704A
:1021C0002B70204638BD30B1002CFAD00124287085
:1021D000F7E70024F5E70446F3E700002DE9F843AC
:1021E0000026D0F8008005460C468E76836B002BC7
:1021F0004AD098F80030042B4BD13346354640275F
:1022000020E0B7F5187F80F0C480F90606F10106DA
:1022100008BF0237D05B02372BB900F5205292B2CB
:10222000B2F5006F0DD305F11A01C5F1FF0240EAC6
:1022300003402144FFF7B6FF002800F0AA800544C0
:1022400000200346D8F8102092F82310B142D8D8C5
:10225000002B40F09E80002D00F09B800023254441
:10226000AB766373D8F81020137903F03701DB06DF
:1022700021730BD402F13800FFF704FFC4E9000119
:1022800093896381D3892381BDE8F88300200146C7
:10229000F4E7C36C01335ED1EA6B00232E26551E92
:1022A000184615F8011F013020290CD0052908BF58
:1022B000E521092804D10B2B9EBFE71801337E735B
:1022C000E718013379730B28EBD1E118002048732C
:1022D000A17E00294BD1002B40D06FF00C0604F1F9
:1022E0000D000825361B331810F8011B002938D0C3
:1022F0002E298BB24AD0A3F14101192903D8117BB1
:102300000D4200D020330373EDE7B9F1000F05D182
:1023100000F520539BB2B3F5006F0BD307F11A0100
:10232000C7F1FF0240EA09402144FFF73BFF48B1F3
:102330000744002002368146D8F80C30985B00280C
:10234000E3D13846B9F1000F4FF0000218BF00206A
:1023500023189A76A0E7B1463746EDE73F23A376E8
:102360000123234400219976137B03B96373D37A45
:1023700002F11C0003F03F0323730023FFF780FEEC
:1023800020606360D38A6381138B7CE710250B4642
:10239000B9E73F230125A37660E7000038B505467D
:1023A000002435F8020B08B9204638BD02F0EEF8DB
:1023B0006308C2B203EBC43312FA83F39AB2C0F3D8
:1023C000072303EB520303EBC2339CB2E9E700009F
:1023D00037B5C37804461BB90025284603B030BD85
:1023E00000F14C01826C01234078019103F0C8FF99
:1023F000054680B9A36BE070A06C226BC31A9342B0
:10240000EAD2A3780199022BE6D102440123607835
:1024100003F0B6FFE1E70125DFE7000038B5836C84
:1024200005460C468B4210D0FFF7D2FF60B922461A
:10243000012305F14C01687803F07EFF00281CBFE2
:102440004FF0FF340120AC6438BD0020FCE70000F1
:1024500038B500230446C3704FF0FF338364FFF7A1
:10246000DDFF00284BD1B4F84A524AF655239D426D
:1024700007D10B22254904F14C0006F015FA00287B
:102480003FD094F84C30EB2B03D01833DBB2012B48
:102490002ED84AF655239D4206D108221C4904F144
:1024A0009E0006F001FA48B3B4F85730B3F5007F48
:1024B0001ED194F85930DBB15A1E1A4218D1B4F823
:1024C0005A30ABB194F85C30013B012B10D8B4F812
:1024D0005D306BB1B4F85F307F2B06D804F16C002F
:1024E000FFF7CEFDB0F5803F02D3B4F8623053B9A8
:1024F0004AF6552085420CBF0220032038BD042037
:10250000FCE70120FAE70020F8E700BF748A000822
:10251000808A000802392DE9F04701F007044FF0E6
:10252000010A466C05460AFA04F41746984606EB7B
:102530001136C1F3C809E4B2314628460136FFF727
:102540006DFF18B10120BDE8F087994605EB09023F
:1025500092F84C30234214BF01210021414513D091
:102560006340013F82F84C3085F803A0EBD0640053
:1025700014F0FF04EAD109F1010301244FF000092E
:10258000B3F5007FE1D1D7E70220DCE7012902465D
:10259000F8B50C4640F28C800668F36A8B4240F234
:1025A00087803378013B032B00F28280DFE803F061
:1025B0000229384B04EB5405B16B304601EB552131
:1025C000FFF72CFF10B14FF0FF30F8BD6F1CC5F3C3
:1025D0000805B16B3046354401EB572195F84C5056
:1025E000FFF71CFF0028EED1C7F30807E3073E44BE
:1025F00096F84C0045EA00204CBF0009C0F30B00E0
:10260000E3E7B16B304601EB1421FFF707FF002829
:10261000D9D1640004F4FF742644B6F84C00D4E722
:10262000B16B304601EBD411FFF7F8FE0028CAD198
:10263000A40006F14C0004F4FE742044FFF720FDD2
:1026400020F07040C1E7D0E90430D57953EA0001A9
:1026500001D0916801B95DBB9168022DA4EB010125
:102660000DD1013B728940F1FF305B0A43EAC05350
:10267000B3FBF2F399421BD81CD0601CA5E7032DD5
:1026800002D193698B42F8D8D3699BB9B16B3046BC
:1026900001EBD411FFF7C2FE002894D1A0004C3604
:1026A00000F4FE703044FFF7EBFC20F000408CE7B4
:1026B00001208AE76FF0004087E70000F8B5066860
:1026C00004460D463378042B0CBF4FF080524FF474
:1026D00000128A4201D80220F8BDCA06FBD18268E6
:1026E0000163D2B9022B13D83389B3EB551FF2D94A
:1026F000F36BA363A36B6263002BECD003EB552356
:102700004C36C5F308050020A3633544E563E3E7D1
:10271000F36BC271002BE7D01A4677897F02BD4266
:10272000114604D23046FFF7C9FCA063E2E7204619
:10273000FFF72CFF431C024606D00128CBD9F36AD1
:102740008342C8D9ED1BEAE70120C5E701292DE93D
:10275000F04706460C46174608D9C36A8B4205D98E
:102760000378022B62D003D8012B22D0022552E03D
:10277000033B012BFAD8816B01EBD411FFF74EFE1E
:102780000546002847D1A40006F14C0304F4FE746A
:102790001C443378042B07D0204627F07047FFF7FE
:1027A0006FFC00F07040074339462046FFF76EFC8F
:1027B0002FE001EB5108816B01EB5821FFF72EFE52
:1027C000054640BB14F0010406F14C0908F1010A6A
:1027D000C8F3080808BFFBB230461FBF19F808301D
:1027E00003F00F023B0103F0F00318BF134309F895
:1027F00008300123B16BF37001EB5A21FFF70EFE95
:10280000054640B9CAF3080A44B1C7F3071709F8E7
:102810000A700123F3702846BDE8F08719F80A30E2
:10282000C7F3032723F00F031F43F0E7816B01EB8E
:102830001421FFF7F3FD05460028ECD1640006F1F2
:102840004C0304F4FF741F551919C7F307274F7081
:10285000DFE70000F8B504460E461746E3690BB9FA
:102860001846F8BD012BA6EB0305206814BFAA1C6F
:102870003A46691CFFF76AFF0028F2D1E369013B81
:10288000E361EBE701292DE9F84306460C461746BC
:10289000056802D80220BDE8F883EB6A8B42F9D9BB
:1028A0007AB9A14621463046A046FFF76FFE04469E
:1028B000B0B92B78042B02D1002F43D1F77100203F
:1028C000E9E72B78042B02D1C379022BE9D04FF032
:1028D000FF3239462846FFF739FF0028E1D0DAE712
:1028E0000128D7D0421C01D10120D4E72B78042B3A
:1028F00019D1EA6AAB69023A93421CD308F101028A
:10290000A2420CD02B78042B08D10023A2EB0902A1
:1029100049462846FFF7FEFD0028BCD1A146EB6AD8
:10292000A342BFD8C5E7002241462846FFF70EFF65
:102930000028DED0AFE70133AB612B7943F0010310
:102940002B71DBE7F3798BB9B468BC4202D1022367
:10295000F371B4E721463046FFF718FE012899D9F4
:10296000431CC1D001348442EFD0A8E7032BA6D189
:10297000B368BB42A3D8B2691344BB429FD3E6E716
:1029800070B5C3790446032B06D181688369CD18DD
:10299000A94203D10023E371002070BD4E1C2068C2
:1029A0003246FFF7D3FE0028F7D13146F0E70000AA
:1029B0002DE9F74305460191FFF70AFD044600287B
:1029C00049D105F14C09019928464FF40072FFF7EF
:1029D00075FB2146A86407464846FFF739FA6C891B
:1029E0006402B4F5004F28BF4FF40044B4F5007FF3
:1029F0002FD9204604F038F9804630B12246002114
:102A0000640A0026FFF724FA09E06408EEE723468B
:102A1000BA194146687803F0B3FC18B926446B89AB
:102A20009E42F4D3404604F02FF96889801B18BFFA
:102A3000012003B0BDE8F08301366B899E42F4D2D9
:102A40000123BA194946687803F09AFC0028F3D0AC
:102A5000EBE70026F1E70120EBE70000F8B50446BC
:102A6000FFF7B6FC0546002842D12378032B37D167
:102A70002779012F34D104F14C0601464FF400723E
:102A80003046FFF7E5F955234122722184F84A3296
:102A9000AA2304F50D7084F84F2084F84B3252239A
:102AA00084F8301284F84C3084F84D30612384F877
:102AB000311284F84E3084F83332A16984F832221E
:102AC000FFF7E4FA616904F50E70FFF7DFFA626B55
:102AD0003B46314601326078A26403F051FC257117
:102AE00000226078114603F06FFC003818BF012007
:102AF000F8BD000000232DE9F0430B6085B00F46C0
:102B00001546FFF71BFB061EC0F2B281804B53F83F
:102B10002640002C00F0AE813C6005F0FE052378D5
:102B20006BB1607803F006FCC70708D41DB110F044
:102B3000040500D00A25284605B0BDE8F08300232F
:102B4000F0B22370607003F0E1FBC10700F19481E3
:102B50000DB14207EED400212046FFF779FC022890
:102B600040F099806E4604F2122304F2522132465C
:102B700018461033FFF784FA42F8040B8B42F7D162
:102B8000002556F8041B00297DD02046FFF760FC85
:102B9000012879D80128A26C40F0C08004F15703C5
:102BA00004F18C0113F8015B002D7BD18B42F9D12C
:102BB000B4F8B430B3F5807F74D194F8B830092BF1
:102BC00070D104F19400FFF75DFA4FF0FF3317184E
:102BD00041F10001BB4275EB010363D304F1A00096
:102BE000FFF74EFA94F8BA302063012BA37059D145
:102BF00094F8B99003FA09F91FFA89F36381002B5D
:102C000050D0444B04F1A800FFF73AFA0646984228
:102C100048D8831C626304F1A400E362FFF730FA32
:102C200000EB020804F19C00C4F84080FFF728FA8A
:102C300010441FFA89F2A06306FB02F313EB0803AA
:102C400045EB05029F4271EB02032BD32E4604F1A4
:102C5000AC00FFF715FAE06365B96389B34221D987
:102C6000E16B2046FFF72AFA81192046FFF7D6FBD1
:102C700098B90136631993F84C30812B14D0203564
:102C8000C5F30805E8E703200135042D7FF479AF8B
:102C9000042807D101E0042801D101254BE70128D0
:102CA0007FF678AF0D2546E705F1140004F14C06D8
:102CB0003044FFF7E5F901280546F3D9E36A83427A
:102CC000F0D96189821E236C02FB01336364A16B1E
:102CD000204601EBD511FFF7A1FB0028DDD105F05F
:102CE0007F0006EB8000FFF7CBF9431C03D00135D2
:102CF000A842ECD0D6E70425C4E90500064A2570B1
:102D000000251388E56101339BB21380E38012E74D
:102D100014360020FDFFFF7F18360020B4F857302E
:102D2000B3F5007FBED1B4F8626026B904F170003B
:102D3000FFF7A6F9064694F85C302663591EA37087
:102D40000129AFD894F859506581002DAAD0691E89
:102D50002942A7D1B4F85D8018F00F0FA4F80880BD
:102D6000A0D1B4F85F0018B904F16C00FFF788F93E
:102D7000B4F85A10002995D006FB03FE01EB181C8D
:102D8000F44460458ED3A0EB0C00A842B0FBF5F3F1
:102D900088D33E48834285D84FF6F57083426DD97B
:102DA00003259F1C114402EB0C03032DE7626263B1
:102DB000A16323644CD1B4F8763053EA08037FF45E
:102DC00071AFBB0004F17800FFF75AF9E06303F23A
:102DD000FF13B6EB532FFFF465AF4FF0FF33032D16
:102DE000C4E905334FF08003237187D1B4F87C30F8
:102DF000012B83D1511C2046FFF710FB00287FF4E4
:102E00007DAFB4F84A224AF6552320719A427FF4E6
:102E100075AF1F4B04F14C00FFF732F998427FF475
:102E20006DAF03F1FF5304F50C70FFF729F903F5BB
:102E30000053203398427FF461AF04F50D70FFF723
:102E40001FF9A06104F50E70FFF71AF9606155E7EC
:102E5000B8F1000F3FF426AF7144022D4FEA47034B
:102E6000E1631EBFD91907F0010303EB5103AEE77D
:102E70000B2560E60C255EE603255CE640F6F5755D
:102E8000AB428CBF022501258BE700BFF5FFFF0F8A
:102E9000525261412DE9F84F07460568884649B905
:102EA0006E69C6B1EB6AB34298BF0126AB69A3B99C
:102EB000002405E0FFF76AFB0128044603D801243B
:102EC0002046BDE8F88F421C00F0D280EB6A8342B6
:102ED000F6D84646EAE70126E8E72A78EB6A042AAC
:102EE00040F08380A6F1020A023B4FF0010B9A45A5
:102EF00028BF4FF0000AD146696C284601EB193112
:102F0000FFF78CFA00283BD109F00703EA6AC9F3FE
:102F1000C8010BFA03F3901EDBB26A184C4609F1A4
:102F2000010992F84C20814502EA030233BF5B009D
:102F300000234FF40071DBB228BF9946B2B90234C6
:102F4000631E0333BCD80123214628461A46FFF7E7
:102F5000E1FA0228B3D0012800F08A80B8F1000F0E
:102F600013D10223FB710028A9D130E0CA450AD051
:102F7000002BD2D10131B1F5007FBDD20123CCE7C6
:102F80004FF0FF34DCE70024DAE7FB79022B07D1AE
:102F9000731CA342E7D0BB68F31ABB610323FB7128
:102FA00008F10102FB69A24205D113B10133FB61B3
:102FB000D9E70223FBE70BB90123FB612246414617
:102FC0003846FFF747FC00284FD10123FB61EA6A2E
:102FD000AB69023A6C6193429CBF03F1FF33AB6172
:102FE0002B7943F001032B716AE7464514D1741C19
:102FF0003846A34298BF02242146FFF7C7FA0128AA
:103000003FF45DAF431C33D0E0B16B69012B03D9B2
:10301000EA6A934238BF1E4634460134EB6AA34243
:1030200003D8012E7FF644AF022421463846FFF72D
:10303000ADFA48B101283FF442AF013018D0B44294
:10304000EBD135E7002CE7D04FF0FF322146284680
:10305000FFF77CFB48B9B8F1000FB8D022464146D3
:103060002846FFF773FB0028B1D001287FF427AF73
:103070004FF0FF3424E700002DE9F84306680446CA
:10308000076B894633782037042B0CBF4FF08053F1
:103090004FF40013BB429CBF00238363836B73B167
:1030A000C7F30808B8F1000F3CD10133416B8363CB
:1030B00039B93389B3EB571F34D80023A3630420F5
:1030C0000AE07389013B13EA57232BD1FFF75EFA1D
:1030D0000128054602D80220BDE8F883421C01D130
:1030E0000120F9E7F36A834216D8B9F1000FE4D062
:1030F000616B2046FFF7CEFE0546C8B10128EAD035
:10310000431CEDD001463046FFF752FC0028E7D1C2
:10311000E37943F00403E371294630466563FEF723
:10312000CDFFA0634C36002027634644E663D3E717
:103130000720D1E7F8B50E46002104460768FFF7DF
:10314000BDFA98B90546A16B3846FFF767F968B92B
:103150003A78E36B042A1B780CD11B060ED5054682
:1031600001212046FFF788FF0028ECD0042808BF83
:10317000072006E0E52B01D0002BF0D10135B54248
:10318000EED1F8BDC16C4B1C2DE9F0410446056839
:10319000066B1FD1E5274FF00108A16B2846FFF70A
:1031A0003DF998B92A78E36B042A09BF1A781F7091
:1031B00002F07F021A7085F80380236BB3420DD2B0
:1031C00000212046FFF758FF0028E6D0042808BF5A
:1031D000022003E0FFF772FA0028DBD0BDE8F0819F
:1031E0002DE9F04105460068A96B0669FFF716F95D
:1031F000044620B9EB6B1A78852A03D002242046B6
:10320000BDE8F081324603F1200153F8040B8B42F4
:1032100042F8040BF9D1777801377F01A7F16003F9
:10322000B3F5007FEAD800212846FFF725FF0428E0
:103230000446E3D00028E2D1A96B2868FFF7EEF836
:1032400004460028DBD1EB6B1A78C02AD6D106F1F0
:10325000200203F1200153F8040B8B4242F8040BC7
:10326000F9D196F823300F222C33B3FBF2F3B7EBEE
:10327000431FC3D34FF0400800212846FFF7FCFE50
:1032800004280446BAD00028B9D1A96B2868FFF7F2
:10329000C5F804460028B2D1EB6B1A78C12AADD12B
:1032A000B8F5187F09D206EB080203F1200153F8A4
:1032B000040B8B4242F8040BF9D108F12008474572
:1032C000DAD8B8F5187F9AD83046FEF71FFF738812
:1032D000834294D092E700000B68002210B503608F
:1032E00004460B6A83604B6AC261C37123F0FF031B
:1032F000896AC0E90432C164FFF7E0F920B92046C9
:10330000BDE81040FFF76CBF10BD0000F8B50368C2
:10331000054601271C692046FEF7F8FEA070000A4A
:103320006678E0702846E96CFFF7C8F920B10228FA
:1033300028BF0220C0B2F8BDA96B2868FFF76EF85D
:103340000028F4D1EB6B04F1200254F8041B9442E2
:1033500043F8041BF9D12B68DF70002EE7D0002161
:103360002846013EFFF788FEE0E700002DE9F8431C
:103370004FF0FF0806460768042445464FF6FF79DC
:10338000B16B11B9002C73D063E03846FFF746F8F3
:10339000044600285DD1F06B0378002B6ED03A789C
:1033A000042A11D1852B4DD1336B3046F364FFF7DE
:1033B00017FF044600284CD13B691B7903F03F03FB
:1033C000B3712046BDE8F883C27AE52B02F03F02D4
:1033D000B27143D02E2B41D022F0200108293DD0DC
:1033E0000F2A40D1590637D503F0BF05336B90F84B
:1033F0000D80F364437B434530D1428B72BB03782D
:103400000D21FC6823F04003DFF874E0013B4B43DF
:1034100001211EF801CB30F80CC009B3FF2B1DD8D9
:1034200024F813C06146013301320D2AF1D102782C
:10343000520605D521B1FF2B10D8002224F8132005
:10344000013DEDB200213046FFF716FE044600288C
:1034500096D00023B363B4E7AB42CBD0FF25F1E7AE
:10346000CC45E1D0FAE72DB9FEF740FE404501D149
:103470000024A6E74FF0FF33F364A2E70424E8E753
:103480001C8B00082DE9F04F002187B00446D0F8CE
:103490000090FFF713F9804670B999F80030042BBB
:1034A00033D1D9F80C00FEF779FF07462046FFF725
:1034B0005DFF054620B18046404607B0BDE8F08F6D
:1034C000D9F810309A8CBA42F0D193F823B0402644
:1034D0005D4506D1D9F80C3033F81530002BE5D115
:1034E000EAE7F106D9F8103008BF0236985B01F020
:1034F0004DF8D9F80C30824633F8150001F046F843
:103500008245D3D102360135E2E74FF0FF0A4FF092
:10351000FF3B5546C4F84CB0A16B4846FEF77EFF12
:1035200000285CD1E66B3778002F77D0F27AE52F50
:1035300002F03F03A37103D0120704D50F2B04D070
:10354000C4F84CB04FE00F2B54D194F84B305806D0
:103550003FD4790645D5236B07F0BF0796F80DA039
:10356000E364737B53453ED1738B002B3BD135789D
:103570000121D9F80C3005F03F0501930D23013DE1
:103580005D43284B13F8012BB25A71B3FF2D0593FD
:1035900029D81046049200F0F9FF6B1C03900293A7
:1035A000019B33F8150000F0F1FF039981421AD115
:1035B000049A029D1146059B1B4A9342E2D133783F
:1035C0005A0604D519B1019B33F815305BB97D1E3D
:1035D000EDB200212046FFF74FFD00289CD0804629
:1035E0006AE7BD42BDD0FF25F3E74FF6FF70824288
:1035F000E2D0F8E72DB93046FEF778FD50453FF4AC
:103600005BAF94F84B30DB079AD40B2204F14001F6
:10361000304605F049F9002892D14DE74FF00408F3
:103620004AE700BF1C8B0008298B00082DE9F04FEA
:1036300090F84BB099B004461BF0A00540F06881AB
:103640000668F26832F81530002B4AD13378042B23
:1036500040F087800F230E352046B5FBF3F5A91CFB
:10366000FFF768FD8146002877D1236B0135A3EB76
:103670004515E3795A07E56435D523F00403204660
:10368000E371FFF77DF950BB4FF0FF32616B2046CD
:10369000FFF7E0F818BBA3682BB3214604A8FFF797
:1036A0001BFEE0B970894FF40071D4E90423E0FBFC
:1036B00001233069C4E904233830FEF7EFFC306998
:1036C000D4E904232830FEF7E9FCE379326904A841
:1036D00043F0010382F82130FFF718FE18B181464C
:1036E0003BE00135AEE7D6E90354402200212046F5
:1036F000FEF7AEFB8523012140222370C0234FF04B
:10370000C10C04EB010884F8203000231E469E46BD
:10371000571C04F802C0F0B2023204F807E021B1ED
:1037200035F8131009B10133DBB20F0AA15408F8C0
:1037300002700232D706F2D135F813700136002F2D
:10374000E6D184F82330831C28466370FEF726FEFA
:1037500084F82400000A84F82500484619B0BDE822
:10376000F08F04F140070DF1100A1BF0010F97E8EC
:1037700007008AE8070000F0D38040234FF00108DB
:1037800084F84B30BC46F368B8F1050F9AE807009F
:10379000ACE803002CF8022B4FEA12428CF8002010
:1037A00059D9981E424630F8021F002942D10DF126
:1037B0000F0C072102F00F0E914612090EF1300096
:1037C000392888BF0EF1370001390CF8010902D001
:1037D000B9F10F0FEED818AB7E205A1802F8580C2A
:1037E00038460022914206D010F801CB02F1010EBA
:1037F000BCF1200F31D104F13F0C072902F1010285
:1038000097BF18AB20205818013198BF10F8580CFA
:10381000072A0CF80200F0D92046FFF733FE814654
:10382000002878D108F10108B8F1640FAAD14FF04F
:10383000070992E74FF0100C01F0010E49080EEB5A
:103840004202D30344BF82F4883282F02102BCF1E9
:10385000010CF1D1A7E74246A9E77246C2E7216B06
:103860002046A1EB4511FEF729FF814600287FF491
:1038700074AF4FF6FF783846FEF738FC0190A16B25
:103880003046FEF7CBFD814600287FF466AFE36B40
:10389000E9B2019A4FF00D0CD6F80CE05A734FF0D4
:1038A0000F02DFF8E0A0DA724A1E18730CFB02F276
:1038B00084469876D87640451AF8019B0CF1010CA5
:1038C00018BF3EF8120003EB090B18BF013203F8D2
:1038D00009004FEA1029002808BF4046BCF10D0F2F
:1038E0008BF80190E7D1404502D03EF812200AB98A
:1038F00041F040011970012300212046F370FFF7C9
:10390000BBFB814600287FF428AF013DB7D11BE007
:103910004FF0060921E704287FF41FAF84F84BB06D
:103920001BF0020F20461BBF0C350D210125B5FBF6
:10393000F1F518BF01352946FFF7FCFB8146002849
:103940007FF40BAF013D8AD1A16B3046FEF766FDD7
:10395000814600287FF401AF01462022E06BFEF78C
:1039600077FAE36B03CF18605960BA7839889A7296
:10397000198194F84B30E26B03F0180313730123A1
:10398000F370EAE61C8B000810B504460A46343092
:10399000FEF776FB886004F13800FEF773FBC2E99E
:1039A000040194F8213003F00203D3710023D361A2
:1039B00010BD000003284B8B04BF8A8A43EA0243F0
:1039C000184670472DE9F04F0B7899B004468946A8
:1039D0002F2BD0F800B001D05C2B09D14A461378C8
:1039E000914601322F2BFAD05C2BF8D0002301E056
:1039F000DBF81C30A3600023E3619BF80030042B4C
:103A00001ED1A368E3B1DBF82030214604A823626D
:103A1000DBF824306362DBF82830A362FFF75CFC3C
:103A20000346002854D1DBF8102002F13800FEF7DD
:103A300027FBC4E9040392F8213003F00203E37189
:103A400099F800301F2B00F2358180230021204699
:103A500084F84B3019B0BDE8F04FFEF72FBE494651
:103A60000B78894601312F2BFAD05C2BF8D01F2B15
:103A70008CBF00250425012F2FD113882E2B31D187
:103A8000002322F8173004F140029F428CBF2E2100
:103A9000202101330B2B02F8011BF6D145F0200544
:103AA000204684F84B50FFF7EDFC94F84B3000288B
:103AB00000F0E78004280BD1990603F0040240F1DE
:103AC000DC80002A00F0F6808023002084F84B3050
:103AD00019B0BDE8F08F0425CDE7022F02D153883D
:103AE0002E2BCAD0911E87BB002322F81730002F3F
:103AF00000F0118132F81300194601332028F9D063
:103B000009B92E2801D145F00305901E30F8173071
:103B10002E2B01D0013FF9D14FF020334FF0000A96
:103B20006364D0462364C4F847300823481C32F845
:103B300011600090F6B1202E03D02E2E0DD1B84288
:103B400010D045F003050099F0E731F81730202B2D
:103B500001D02E2BC8D1013FC5E79A4505D2009967
:103B6000B9423BD10B2B30D101E00B2B27D145F0D3
:103B700003050B2394F84020E52A04BF052284F8AE
:103B80004020082B04BF4FEA88085FFA88F808F045
:103B90000C030C2B03D008F00303032B01D145F0D9
:103BA0000205A8073FF57CAF18F0010F18BF45F0DC
:103BB000100518F0040F18BF45F0080570E70099CC
:103BC000B94202D045F00305D4D84FEA88080B2348
:103BD0004FF0080A00975FFA88F8B4E77F2E15D9EE
:103BE000304640F25231CDE9022345F00203019301
:103BF00000F098FC10F0800F0646DDE9022316D095
:103C000000F07F0646498E5D019D46B3314645482A
:103C1000CDE9012304F072FEDDE90123F8B9A6F134
:103C2000410189B219291ED848F0020810E0FF2886
:103C3000EAD9591E8A4503D345F003059A4682E71F
:103C400004EB0A01000A0AF1010A019D81F8400013
:103C500004EB0A010AF1010A81F8406073E745F0BC
:103C600003055F26F4E7A6F1610189B219299EBF19
:103C7000203E48F00108B6B2EAE7002A08BF052056
:103C800026E75A073FF524AFA379DB0645D59BF815
:103C90000000042835D1A3682146E2792362236914
:103CA000DBF8100023F0FF0313436362E36CA362AD
:103CB000FFF76AFE23680027DA6819F8010B00286D
:103CC0003FF409AF40F25231009200F04BFC054640
:103CD00008B31F28009A7FF6FEAE2F283FF4BFAE30
:103CE0005C283FF4BCAE7F2805D801460E4804F09E
:103CF00005FE009A78B9FF2F0DD022F81750013732
:103D0000DBE7216B0BF14C03C1F308011944FFF70A
:103D100051FEA060CEE70620DAE60520D8E600BF17
:103D20009C8A0008958A00088C8A00081FB5CDE996
:103D3000001003A814460391FEF700FA002815DBD3
:103D40000B4A52F820300BB100211970019B0BB1C6
:103D50000021197042F820302CB1002201A96846D8
:103D6000FEF7C8FE0446204604B010BD0B24FAE757
:103D7000143600202DE9F04798B090460546019191
:103D8000002800F0528102F03F0603A901A8324644
:103D9000FEF7B0FE002840F04681039B4FF48C6094
:103DA000049302F061FF0746002800F04081039B66
:103DB00000F500720199D86004A81A61FFF702FEAD
:103DC000044620B99DF95B30002BB8BF062418F0DB
:103DD0001C0F00F0CD80002C4CD0042C40D104A846
:103DE000FFF724FC044600283AD146F00806039B5E
:103DF0001A78042A40F08380186929462B60FFF75F
:103E0000C3FD039B1E22002118690230FEF720F833
:103E1000039C00211A2220692630FEF719F8236935
:103E200020221A71246902F059FF01460122083448
:103E30002046FEF72BF9039B04A81B6983F8212079
:103E4000FFF764FA044658B9A96801B30246284648
:103E5000FEF718FDAB68039A0446013B5361B4B109
:103E6000384602F011FF0CB100232B60204618B039
:103E7000BDE8F0879DF8163013F0110F40F08480F4
:103E800018F0040F40F0C98018F0080FAFD1039A62
:103E900031071399936C48BF46F04006E964AB6460
:103EA0001078042872D1069B9DF817102B62089B8E
:103EB000106923F0FF030B4329466B62179BAB622B
:103EC000FFF762FDDDF80CA00024002205F1500888
:103ED000BAF8063021464046C5F800A0AB80002362
:103EE00085F8306085F831406C64C5E90E234FF4E5
:103EF0000072FDF7ADFFB20653D40024B0E702F024
:103F0000EDFE0146009013980E30FEF7BFF81398AF
:103F100000991630FEF7BAF8039C13992078FFF742
:103F200049FD202300228046CB7220461399FEF7DC
:103F3000D1F8139B002201211A775A779A77DA7702
:103F4000039BD970B8F1000FA1D0414604A8D3F863
:103F50004890FEF797FC0446002881D14946039813
:103F6000FEF75CFA039B044608F1FF30586176E7E0
:103F7000002C7FF475AF9DF81630DC064FD418F096
:103F8000020F84D0D80782D5072469E7FFF712FD16
:103F90000023A86001F11C00FEF772F86B61286134
:103FA00090E7D5E9046956EA0903A6D0BAF80AA051
:103FB000A9684FEA4A2AC5E90E69B24574EB0903BC
:103FC0001BD300242964002C7FF44AAFC6F30803F6
:103FD000002B92D0039C2046FEF770F808B3760AB7
:103FE0000123414646EAC95682196A64607802F0A4
:103FF000A3F9041E18BF012432E72846FEF7C6FACB
:10400000B6EB0A06014669F10009012803D9431CF1
:10401000D3D10124D6E70224D4E7082420E70424DE
:104020001EE702241CE704461EE709241EE71124AC
:104030001CE700002DE9F04F994685B00023884623
:1040400003A90446C9F800301646FEF791F8054664
:1040500080BB94F831506DBB94F8303013F00103FD
:10406000009300F0A68004F1500AD4E90432D4E9A8
:104070000E011B1A62EB0102B34272F1000238BF5B
:104080001E46BEB1D4E90E10C1F30803002B40F068
:104090008280039B5A894B0A013A43EAC0531A4073
:1040A0001BD151EA000309D1A06801280DD80225CF
:1040B00084F83150284605B0BDE8F08F216C2046C9
:1040C0000192FEF763FA019AEFE7431C04D1012342
:1040D000009D84F83130EDE72064DDF80CB0216CF0
:1040E0005846FDF7EBFF0028E1D0B6F5007F02EB64
:1040F000000731D3BBF80A1002EB5620730A88423E
:104100009BF8010088BF8B1A3A464146019302F0A2
:1041100013F90028DBD194F93020019B002A0BDA37
:10412000606CC01B984207D24FF40072514608EBF6
:104130004020FDF767FE019B5F02D9F80030F61BB7
:10414000B8443B44C9F80030D4E90E32DB1942F1DF
:104150000002C4E90E3294E7626CBA421AD094F9B4
:104160003030002B0DDA012351469BF8010002F09C
:1041700007F90028ABD194F8303003F07F0384F8BE
:104180003030039801233A465146407802F0D4F883
:1041900000289CD16764A16B4046C1F30801C1F5BA
:1041A00000775144B74228BF37463A46FDF72AFE0A
:1041B000C3E707257EE7000070B596B00E460022E3
:1041C000019002A901A8FEF795FC0446E0B94FF45E
:1041D0008C6002F049FD0546D8B1029B00F50072E3
:1041E0000199D86002A81A61FFF7ECFB044640B9B8
:1041F0009DF95330002B0ADB1EB1314602A8FDF7B2
:10420000EDFF284602F040FD204616B070BD0624A2
:10421000F7E71124F8E7000070B5B8B0022201906A
:1042200003A901A8FEF766FC044608BB039B4FF4F4
:104230008C60109302F018FD0546002866D0039BA1
:1042400000F500720199D86010A81A61FFF7BAFB57
:10425000044650B99DF88B30980655D4190653D4AE
:104260009DF84630DA0706D50724284602F00CFDF3
:10427000204638B070BD039B04931878042814D1ED
:1042800004A91869FFF780FB069E9DF84630DB06FF
:1042900010D410A8FEF776FF04460028E5D156BBDF
:1042A0000398FEF7DBFB0446DFE71F99FFF782FB6D
:1042B0000646EAE7039BDA69B242D5D0249300218F
:1042C000269624A81B78042B01BFDDE90823CDE93D
:1042D00028239DF817308DF89730FEF7EFF9044644
:1042E0000028C2D124A8FFF741F804460028BBD01B
:1042F0000428BAD1CDE70246314604A8FEF7C2FA37
:1043000004460028B1D1CBE70624AEE71124AFE77D
:10431000F0B5BDB0CDE900106846FDF70FFF0222F1
:1043200003A901A8FEF7E6FB0446002841D1039B40
:104330004FF48C60149302F097FC0546002800F0BF
:10434000EE80039B00F5007214AE0199D8601A61EB
:104350003046FFF737FB044640BB9DF89B3013F017
:10436000A00F40F0D880039B009F1A78042A68D1E0
:104370001B6904AC03F1400C1868083353F8041CA3
:104380002246634503C21446F6D15022314628A87E
:10439000FDF738FD394628A8FFF714FB044600282E
:1043A0004CD12A9A169B9A4206D00824284602F03D
:1043B0006BFC20463DB0F0BD349A209B9A42F4D16C
:1043C00028A8FFF733F904460028EFD1039B04AF78
:1043D0001B6993F801E093F823C09C8C3A4608339C
:1043E00003CAB24243F8080C43F8041C1746F5D13F
:1043F000039B28A81B6983F801E0039B1A6982F8D4
:1044000023C01A6982F82440240A82F825401A69D8
:104410001379D9065CBF43F020031371FEF776FFD2
:1044200004460028C2D13046FEF7ACFE0446002800
:10443000BCD10398FEF712FB0446B7E70428B5D1B8
:10444000BEE7239A04AB02F1200C1068083252F840
:10445000041C1C46624503C42346F6D15022314653
:1044600028A8FDF7CFFC394628A8FFF7ABFA044689
:1044700000284CD12A9A169B9A4296D1349A209BB6
:104480009A4292D128A8FFF7D1F8044600288DD18E
:1044900037990DF11D030DF12D0001F10D0253F8B7
:1044A000044B834242F8044BF9D11888012710804D
:1044B0009B7893709DF81B30039CDA0658BF43F03D
:1044C0002003CB72E770CB7ADB06ACD5169A2A9B19
:1044D0009A42A8D02078FFF76DFA01462046FDF7F2
:1044E000EDFD0146C8B12046FDF798FF04460028BF
:1044F0007FF45CAF039890F86D302E2B93D12A9AFD
:1045000000F16C01FDF7E6FD039BDF708BE70428EB
:104510007FF44CAFB6E7062448E7022446E71124AF
:1045200047E700007F2810B501D880B210BDB0F574
:10453000803F13D240F2523399420FD108490022F2
:1045400031F8024B93B2844203D103F18000C0B230
:10455000ECE70132802AF3D11346F6E70020E5E7C5
:10456000DC8D00087F280DD940F25233994208D1E2
:10457000FF2806D800F10040034B803833F81000C4
:1045800070470020704700BFDC8D0008B0F5803F09
:10459000F0B522D21F4A83B21F49B0F5805F28BF11
:1045A0000A46141D34F8042C2146AAB1934213D3B1
:1045B00034F8025C2E0AEFB252FA85F5A84222DAEC
:1045C000082E09D8DFE806F0050A10121416181A8A
:1045D0001C00801A34F810301846F0BD981A00F00C
:1045E00001001B1A9BB2F7E7103BFBE7203BF9E702
:1045F000303BF7E71A3BF5E70833F3E7503BF1E7C9
:10460000A3F5E353EEE70434002ECBD101EB4702D0
:10461000C7E700BF2C8B0008208D000808B5074BAA
:10462000074A196801F03D01996053680BB1906821
:104630009847BDE8084002F047BD00BF00000240B7
:104640001C36002008B5084B1968890901F03D01A6
:104650008A019A60054AD3680BB110699847BDE892
:10466000084002F031BD00BF000002401C360020AF
:1046700008B5084B1968090C01F03D010A049A605D
:10468000054A53690BB190699847BDE8084002F0AC
:104690001BBD00BF000002401C36002008B5084BBF
:1046A0001968890D01F03D018A059A60054AD369B0
:1046B0000BB1106A9847BDE8084002F005BD00BF85
:1046C000000002401C36002008B5074B074A596815
:1046D00001F03D01D960536A0BB1906A9847BDE87B
:1046E000084002F0F1BC00BF000002401C36002070
:1046F00008B5084B5968890901F03D018A01DA6063
:10470000054AD36A0BB1106B9847BDE8084002F028
:10471000DBBC00BF000002401C36002008B5084B7F
:104720005968090C01F03D010A04DA60054A536B2F
:104730000BB1906B9847BDE8084002F0C5BC00BFC4
:10474000000002401C36002008B5084B5968890D4E
:1047500001F03D018A05DA60054AD36B0BB1106C9C
:104760009847BDE8084002F0AFBC00BF000002401F
:104770001C36002008B5074B074A196801F03D01B7
:104780009960536C0BB1906C9847BDE8084002F0FB
:104790009BBC00BF000402401C36002008B5084B3B
:1047A0001968890901F03D018A019A60054AD36CB4
:1047B0000BB1106D9847BDE8084002F085BC00BF02
:1047C000000402401C36002008B5084B1968090C8B
:1047D00001F03D010A049A60054A536D0BB1906DDA
:1047E0009847BDE8084002F06FBC00BF00040240DB
:1047F0001C36002008B5084B1968890D01F03D01F1
:104800008A059A60054AD36D0BB1106E9847BDE8D2
:10481000084002F059BC00BF000402401C360020D2
:1048200008B5074B074A596801F03D01D960536E3E
:104830000BB1906E9847BDE8084002F045BC00BF40
:10484000000402401C36002008B5084B596889094D
:1048500001F03D018A01DA60054AD36E0BB1106F99
:104860009847BDE8084002F02FBC00BF000402409A
:104870001C36002008B5084B5968090C01F03D01B1
:104880000A04DA60054A536F0BB1906F9847BDE890
:10489000084002F019BC00BF000402401C36002092
:1048A00008B5084B5968890D01F03D018A05DA60A9
:1048B000054AD36F13B1D2F880009847BDE808408D
:1048C00002F002BC000402401C36002000230C4908
:1048D00010B51A460B4C0B6054F82300026001EB34
:1048E000430004334260402BF6D1074A4FF0FF33B8
:1048F0009360D360C2F80834C2F80C3410BD00BF16
:104900001C360020DC8E0008000002400F28F8B59D
:1049100010D9102810D0112811D0122808D10F2436
:104920000720DFF8C8E00126DEF80050A04208D9D1
:10493000002653E00446F4E70F240020F1E70724A3
:10494000FBE706FA00F73D424AD1264C4FEA001C2D
:104950003D4304EB00160EEBC000CEF80050C0E95A
:104960000123FBB273B12048D0F8D83043F00103E3
:10497000C0F8D830D0F8003143F00103C0F800315E
:10498000D0F8003117F47F4F0ED01748D0F8D83048
:1049900043F00203C0F8D830D0F8003143F00203EE
:1049A000C0F80031D0F8003154F80C00036823F04F
:1049B0001F030360056815F00105FBD104EB0C0330
:1049C0003D2493F80CC05F6804FA0CF43C60212489
:1049D0000560446112B1987B00F04EFB3046F8BD93
:1049E0000130A3E7DC8E0008004402581C3600208A
:1049F00010B5302484F31188FFF788FF002383F378
:104A0000118810BD10B50446807B00F04BFB0123DC
:104A10001549627B03FA02F20B6823EA0203DAB259
:104A20000B6072B9114AD2F8D81021F00101C2F816
:104A3000D810D2F8001121F00101C2F80011D2F80B
:104A4000002113F47F4F0ED1084BD3F8D82022F069
:104A50000202C3F8D820D3F8002122F00202C3F8E2
:104A60000021D3F8003110BD1C360020004402584C
:104A700008B5302383F31188FFF7C4FF002383F3C5
:104A8000118808BD836CC26A8B42506810B506D984
:104A90005A1E4C0002EB4103B3FBF4F3184410BD63
:104AA00001F001038A0748BF43F002034A0748BFE9
:104AB00043F008030A0748BF43F00403CA0648BF8F
:104AC00043F010038A06426B48BF43F020031343B0
:104AD0004363704710B5074C204600F0F3FC064BCB
:104AE0000022C4E91023054BA364054BE363054B87
:104AF000E36410BDA03600200070005200B4C4046E
:104B0000F4360020F4380020C36A0BB9104BC3629E
:104B10000379012B11D10F4B98420ED10E4BD3F8D4
:104B2000D42042F48032C3F8D420D3F8FC2042F4DD
:104B30008032C3F8FC20D3F8FC30436C00221A65A5
:104B4000DA621A605A605A624FF0FF329A63704715
:104B5000DC8F0008A0360020004402580379012BA6
:104B60001BD0436C00221A65DA621A605A605A62DE
:104B70004FF0FF329A63094B98420ED1084BD3F89D
:104B8000D42022F48032C3F8D420D3F8FC2022F4BD
:104B90008032C3F8FC20D3F8FC307047A0360020E8
:104BA0000044025810B5446C0649FFF76BFF606083
:104BB000236842F2107043F003032360BDE8104005
:104BC00001F01CBA801A06000129F8B5466C0B4F9B
:104BD00009D175680A493D40FFF754FF054345F484
:104BE00080557560F8BD746806493C40FFF74AFF80
:104BF000044344F480547460F4E700BF00ECFFFF0A
:104C000080F0FA0240787D01436C00225A601A60FD
:104C100070470000426C0129536823F4404304D0DC
:104C2000022905D001B95360704743F48043FAE785
:104C300043F40043F7E70000436C41F480519A606D
:104C4000D9605A6B1206FCD580229A637047000027
:104C500010B541F48851446CA260E160616B11F0C1
:104C60004502FBD0A26311F0040203D0FFF718FF46
:104C7000012010BD616910461960FAE710B541F4D2
:104C80008851446CA260E160616B11F04502FBD079
:104C9000A26311F0050203D0FFF702FF012010BD4F
:104CA000616910461960FAE773B5134604460E466B
:104CB000302282F31188426CD26B32B14FF0FF3157
:104CC0004030019301F0A6F9019B606C002202655F
:104CD000C263C262456B15F4807504D185F31188F7
:104CE000012002B070BD4FF0FF31816382F3118863
:104CF000012E06D90C21204602B0BDE87040FFF716
:104D0000BDBF1046EDE7000073B5446C0E460025AC
:104D10000192616BA1632565E562FFF7C1FE012E7B
:104D200007D9019B2A460C2102B0BDE87040FFF76D
:104D3000A5BF02B070BD000010B541F49851446C9D
:104D4000A260E160616B11F04502FBD0A26311F03B
:104D50003F0203D0FFF7A4FE012010BD216A1046D8
:104D60001960E1695960A16999606169D960F4E7E6
:104D70002DE9F74304460191006D01A917469846B5
:104D800002F0CAF8064600284AD0626C2046DDF8D8
:104D900004905568C5F3090501356B00A56CB5FB9A
:104DA000F3F54FF47A73B5FBF3F55D43556200F00C
:104DB0004FFB50BB636C4FF0FF3201254146C3F8F7
:104DC000589020461D659A634FF49572DA6342F25B
:104DD00007029F62DA62E36C0A9AFFF74FFFA0B9FD
:104DE000E26C104B11680B407BB929462046FFF757
:104DF0005BFF054648B92E463A460199206D02F000
:104E0000C3F8304603B0BDE8F0833A460199206DFF
:104E100002F0BAF8E26C01212046FFF775FFF0E7D7
:104E20000126EEE708E0FFFD2DE9F7431F46436C3E
:104E300001924FF47A725D6804468846C5F309050D
:104E400001356E00856CB5FBF6F5B5FBF2F5554303
:104E50005D6200F0FDFA20B10125284603B0BDE8EF
:104E6000F0837E0201A9206D324602F055F8054616
:104E70000028F1D0636C019AD4F84C909A65012215
:104E80001A654FF0FF329A634FF49572DA639E62AF
:104E9000236BDB064B4658BF4FEA4828012F42469A
:104EA0001BD912212046FFF7E9FEC0B9D9F800202E
:104EB000104B13409BB9636C42F293023946204673
:104EC000DA62E26CFFF7F0FE804640B932460199A3
:104ED000206D454602F058F8BFE71121E2E732465F
:104EE0000199206D02F050F8E26C39462046FFF738
:104EF0000BFFB2E708E0FFFD2DE9F3411F46436CCD
:104F000001924FF47A725D6804468846C5F309053C
:104F100001356E00856CB5FBF6F5B5FBF2F5554332
:104F20005D6200F095FA20B10125284602B0BDE887
:104F3000F0817E0201A9206D324602F033F8054669
:104F40000028F1D0636C019A9A6501221A654FF02E
:104F5000FF329A634FF48D72DA639E62236BE66CC4
:104F6000DB06334658BF4FEA4828012F424619D97D
:104F700019212046FFF782FEB0B932680F4B13406B
:104F800093B9636C42F2910239462046DA62E26CD0
:104F9000FFF78AFE064638B901993546206D02F0C2
:104FA0003DF8C2E71821E4E70199206D02F036F8D8
:104FB000E26C39462046FFF7A7FEB6E708E0FFFDA2
:104FC00012F0030F2DE9F04107460C4615461E4628
:104FD00017D00E44B44202D10020BDE8F081012375
:104FE000FA6B21463846FFF71FFF0028F5D1284607
:104FF0004FF40072F96B05F500750134FCF702FF00
:10500000E8E7BDE8F041FFF70FBF000012F0030F23
:105010002DE9F04107460C4615461E4617D00E44B2
:10502000B44202D10020BDE8F08129464FF400725D
:10503000F86B05F50075FCF7E5FE0123FA6B2146D8
:105040003846FFF759FF0028EDD10134E8E7BDE805
:10505000F041FFF751BF000000207047302310B52A
:1050600083F311880024436C40302146DC6300F058
:10507000DFFF84F3118810BD090100F160430122B4
:1050800003F56143C9B283F8001300F01F039A408F
:1050900043099B0003F1604303F56143C3F880219A
:1050A0001A60704700F01F0301229A40430900F183
:1050B00060409B0000F5614003F1604303F56143EC
:1050C000C3F88020C3F88021002380F800337047A4
:1050D0000379052B05BF836A002001204B6004BFC4
:1050E0004FF400730B60704770B55D1E866A04460E
:1050F0000D44B54205D9436B43F08003436301205F
:1051000070BD06250571FFF75BFF05232371F7E7E7
:1051100070B55D1E866A04460D44B54205D9436BE1
:1051200043F080034363012070BD07250571FFF73D
:105130006DFF05232371F7E738B505790446052D82
:1051400005D108230371FFF787FF257138BD0120C2
:10515000FCE700000323F0B5037185B00446FFF7B8
:1051600021FD002220461146FFF766FD4FF4D5725F
:1051700003AB08212046FFF781FD0246B8B90123A1
:105180002363039BC3F30323012B09D103AB372113
:105190002046FFF773FD18B9A44B039A1340ABB137
:1051A00020460125FFF730FD0223237137E103ABD1
:1051B000002237212046FFF761FD28B99B4A039B57
:1051C0001A40002A00F0A78002232363236B03F018
:1051D0000F03022B40F0A9806425954E42F2107017
:1051E00000F00CFF03AB324601212046FFF730FDF3
:1051F0000028D5D1039B002B80F293805A0003D561
:10520000236B43F010032363002204F108030221FF
:105210002046FFF791FD02460028C1D104F1380372
:1052200003212046FFF72AFD0028B9D104F1180513
:10523000A26B092120462B46FFF77EFD0028AFD147
:1052400002ABA26B07212046FFF718FD0646002897
:10525000A6D1236B03F00F03022B40F08F807E2238
:105260007F21284603F07CF8012840F28780E76B15
:1052700042F2107000F0C2FE08234FF4007239466B
:1052800020460096FFF774FD002889D1384603F0C8
:10529000B5F8236BA06203F00F03022B72D103ABAE
:1052A000644A06212046FFF7E9FC002871D15F49D6
:1052B000039B1940B1FA81F149092046FFF784FCAC
:1052C00002AB4FF4007210212046FFF7D7FC0546D1
:1052D00000287FF465AF554E029B33427FF460AFE8
:1052E000236B13F00E0F03F00F0273D0022A7FF42A
:1052F00057AFE36A1978012900F09480022900F081
:105300009380002900F089804B4F2046FFF782FCF4
:1053100003AB3A4676E0114620462263FFF78CFC49
:1053200054E7013D7FF45AAF3AE7444D6426444ABE
:105330003E4F012B18BF154603AB002237212046F4
:10534000FFF79CFC00287FF42BAF039B3B427FF4CC
:1053500027AF03AB2A4629212046FFF779FC002816
:105360007FF41EAF039B002BFFF648AF013E3FF4D6
:1053700017AF42F2107000F041FEDDE7284603F05F
:1053800011F886E77E227F212846E66B02F0E8FFCF
:1053900008B9002191E700234022314620460093BE
:1053A0000623FFF7E5FC0028F3D1B3895BBA9B071E
:1053B000EFD5244B40223146204600930623FFF7C9
:1053C000D7FC0028E5D1317C01F00F010F3918BF5F
:1053D000012172E7E36A1978F9B101297FF4E0AE9F
:1053E0002046FFF717FC03ABA26B37212046FFF7DF
:1053F00045FC00287FF4D4AE039B33427FF4D0AE4B
:1054000003AB022206212046FFF738FC00287FF478
:10541000C7AE039B33427FF4C3AE052323712846F6
:1054200005B0F0BD084F70E7084F6EE708E0FFFDDC
:105430000080FFC00001B9030000B7030080FF50E7
:1054400000001080F1FFFF800001B7030002B703E6
:1054500037B504460C4D01ABA26B0D212046FFF77A
:105460000DFC78B9019B2B420BD1C3F34323042BD2
:1054700008D0053B022B04D84FF47A7000F0BEFD33
:10548000E9E7012003B030BD08E0FFFD70B530232F
:10549000054683F3118803790024022B03D184F39A
:1054A0001188204670BD0423037184F311880226FD
:1054B000FFF7CEFF04462846FFF7A6FB2E71F0E764
:1054C000FFF708BB044B0360012303710023436310
:1054D000C0E90A33704700BFE48F000810B53023DD
:1054E000044683F31188C162FFF70EFB02230020FC
:1054F000237180F3118810BD10B53023044683F367
:105500001188FFF72BFB00230122E362227183F352
:10551000118810BD026843681143016003B1184748
:105520007047000013B5406B00F58054D4F8A438E0
:105530001A681178042914D1017C022911D1197932
:10554000012312898B4013420BD101A94C3002F088
:1055500035FED4F8A4480246019B2179206800F06A
:10556000DFF902B010BD0000143002F0B7BD00003A
:105570004FF0FF33143002F0B1BD00004C3002F0A8
:1055800089BE00004FF0FF334C3002F083BE0000B4
:10559000143002F085BD00004FF0FF31143002F0EE
:1055A0007FBD00004C3002F055BE00004FF0FF32CE
:1055B0004C3002F04FBE00000020704710B500F5DF
:1055C0008054D4F8A4381A681178042917D1017CC2
:1055D000022914D15979012352898B4013420ED1EB
:1055E000143002F017FD024648B1D4F8A4484FF435
:1055F000407361792068BDE8104000F07FB910BDAC
:10560000406BFFF7DBBF0000704700007FB5124B17
:1056100001250426044603600023057400F184027A
:1056200043602946C0E902330C4B029014300193C9
:105630004FF44073009602F0C9FC094B04F6944203
:10564000294604F14C000294CDE900634FF4407305
:1056500002F090FD04B070BD0890000801560008EB
:10566000255500080A68302383F311880B790B3322
:1056700042F823004B79133342F823008B7913B19E
:105680000B3342F8230000F58053C3F8A41802231B
:105690000374002080F311887047000038B5037F41
:1056A000044613B190F85430ABB90125201D0221F6
:1056B000FFF730FF04F114006FF00101257700F0CF
:1056C000DDFC04F14C0084F854506FF00101BDE89A
:1056D000384000F0D3BC38BD10B501210446043079
:1056E000FFF718FF0023237784F8543010BD000023
:1056F00038B504460025143002F080FC04F14C005B
:10570000257702F04FFD201D84F854500121FFF74A
:1057100001FF2046BDE83840FFF750BF90F88030C9
:1057200003F06003202B06D190F881200023212A6A
:1057300003D81F2A06D800207047222AFBD1C0E9CF
:105740001D3303E0034A426707228267C3670120D3
:10575000704700BF3422002037B500F58055D5F8DA
:10576000A4381A68117804291AD1017C022917D1AA
:105770001979012312898B40134211D100F14C0495
:10578000204602F0CFFD58B101A9204602F016FDD7
:10579000D5F8A4480246019B2179206800F0C0F8A2
:1057A00003B030BD01F10B03F0B550F8236085B0B4
:1057B00004460D46FEB1302383F3118804EB8507C0
:1057C000301D0821FFF7A6FEFB6806F14C005B695F
:1057D0001B681BB1019002F0FFFC019803A902F0C5
:1057E000EDFC024648B1039B2946204600F098F89C
:1057F000002383F3118805B0F0BDFB685A69126875
:10580000002AF5D01B8A013B1340F1D104F180023C
:10581000EAE70000133138B550F82140ECB13023ED
:1058200083F3118804F58053D3F8A42813685279C0
:1058300003EB8203DB689B695D6845B10421601856
:10584000FFF768FE294604F1140002F0EDFB204644
:10585000FFF7B4FE002383F3118838BD70470000C2
:1058600001F030BD01234022002110B5044600F8AC
:10587000303BFCF7EDFA0023C4E9013310BD000012
:1058800010B53023044683F311882422416000219F
:105890000C30FCF7DDFA204601F036FD0223002033
:1058A000237080F3118810BD70B500EB81030546AD
:1058B00050690E461446DA6018B110220021FCF738
:1058C000C7FAA06918B110220021FCF7C1FA3146CD
:1058D0002846BDE8704001F01DBE0000836820220C
:1058E000002103F0011310B5044683601030FCF76B
:1058F000AFFA2046BDE8104001F098BEF0B4012593
:1059000000EB810447898D40E4683D43A4694581EB
:1059100023600023A2606360F0BC01F0B5BE00000C
:10592000F0B4012500EB810407898D40E4683D4314
:105930006469058123600023A2606360F0BC01F00C
:105940002BBF000070B502230025044624220370FB
:105950002946C0F888500C3040F8045CFCF778FA0F
:10596000204684F8705001F069FD63681B6823B11C
:1059700029462046BDE87040184770BD0378052BC6
:1059800010B504460AD080F88C30052303704368B4
:105990001B680BB1042198470023A36010BD0000D1
:1059A0000178052906D190F88C20436802701B68A5
:1059B00003B118477047000070B590F87030044686
:1059C00013B1002380F8703004F18002204601F00A
:1059D00051FE63689B68B3B994F8803013F060059A
:1059E00035D00021204602F043F90021204602F084
:1059F00033F963681B6813B10621204698470623D4
:105A000084F8703070BD204698470028E4D0B4F880
:105A10008630A26F9A4288BFA36794F98030A56F41
:105A2000002B4FF0300380F20381002D00F0F28054
:105A3000092284F8702083F3118800212046D4E9DC
:105A40001D23FFF76DFF002383F31188DAE794F835
:105A5000812003F07F0343EA022340F202329342A3
:105A600000F0C58021D8B3F5807F48D00DD8012B38
:105A70003FD0022B00F09380002BB2D104F18802BA
:105A800062670222A267E367C1E7B3F5817F00F096
:105A90009B80B3F5407FA4D194F88230012BA0D134
:105AA000B4F8883043F0020332E0B3F5006F4DD014
:105AB00017D8B3F5A06F31D0A3F5C063012B90D8F0
:105AC0006368204694F882205E6894F88310B4F8E6
:105AD0008430B047002884D0436863670368A367B5
:105AE0001AE0B3F5106F36D040F6024293427FF4CD
:105AF00078AF5C4B63670223A3670023C3E794F886
:105B00008230012B7FF46DAFB4F8883023F00203AC
:105B1000A4F88830C4E91D55E56778E7B4F880300B
:105B2000B3F5A06F0ED194F88230204684F88A3005
:105B300001F0E2FC63681B6813B10121204698471D
:105B4000032323700023C4E91D339CE704F18B0376
:105B500063670123C3E72378042B10D1302383F339
:105B600011882046FFF7BAFE85F311880321636888
:105B700084F88B5021701B680BB12046984794F82D
:105B80008230002BDED084F88B30042323706368CE
:105B90001B68002BD6D0022120469847D2E794F804
:105BA000843020461D0603F00F010AD501F054FD94
:105BB000012804D002287FF414AF2B4B9AE72B4B1B
:105BC00098E701F03BFDF3E794F88230002B7FF477
:105BD00008AF94F8843013F00F01B3D01A062046B2
:105BE00002D502F05DF8ADE702F04EF8AAE794F8AE
:105BF0008230002B7FF4F5AE94F8843013F00F015F
:105C0000A0D01B06204602D502F032F89AE702F037
:105C100023F897E7142284F8702083F311882B4629
:105C20002A4629462046FFF769FE85F31188E9E6F2
:105C30005DB1152284F8702083F31188002120467D
:105C4000D4E91D23FFF75AFEFDE60B2284F87020ED
:105C500083F311882B462A4629462046FFF760FE2B
:105C6000E3E700BF38900008309000083490000847
:105C700038B590F870300446002B3ED0063BDAB2BF
:105C80000F2A34D80F2B32D8DFE803F03731310830
:105C9000223231313131313131313737856FB0F81E
:105CA00086309D4214D2C3681B8AB5FBF3F203FB16
:105CB00012556DB9302383F311882B462A462946A5
:105CC000FFF72EFE85F311880A2384F870300EE06A
:105CD000142384F87030302383F311880023204686
:105CE0001A461946FFF70AFE002383F3118838BDD0
:105CF000C36F03B198470023E7E70021204601F076
:105D0000B7FF0021204601F0A7FF63681B6813B1AD
:105D10000621204698470623D7E7000010B590F8E3
:105D200070300446142B29D017D8062B05D001D883
:105D30001BB110BD093B022BFBD80021204601F00E
:105D400097FF0021204601F087FF63681B6813B1AD
:105D5000062120469847062319E0152BE9D10B238D
:105D600080F87030302383F3118800231A461946D7
:105D7000FFF7D6FD002383F31188DAE7C3689B6938
:105D80005B68002BD5D1C36F03B19847002384F81B
:105D90007030CEE70023826880F8243083691B6866
:105DA00099689142FBD25A68036042601060586063
:105DB000704700000023826880F8243083691B68E4
:105DC00099689142FBD85A6803604260106058603D
:105DD0007047000008B50846302383F3118891F816
:105DE0002430032B05D0042B0DD02BB983F311885D
:105DF00008BD8B6A00221A604FF0FF338362FFF701
:105E0000C9FF0023F2E7D1E9003213605A60F3E7DB
:105E1000034610B51B68984203D09C688A68944278
:105E2000F8D25A680B604A601160596010BD0000DA
:105E3000FFF7B0BF064BD96881F8240018680268E4
:105E400053601A600122D86080F82420FAF7DABA89
:105E5000F83800200C4B30B5DD684B1C87B0044689
:105E60000FD02B46094A684600F09CF92046FFF700
:105E7000E1FF009B13B1684600F09EF9A86A07B0E5
:105E800030BDFFF7D7FFF9E7F8380020D55D0008EF
:105E9000044B1A68DB6890689B68984294BF0020A6
:105EA00001207047F8380020094B10B51C68D868ED
:105EB000226853601A600122DC6084F82420FFF716
:105EC00079FF01462046BDE81040FAF79BBA00BFB3
:105ED000F8380020044B1A68DB6892689B689A4285
:105EE00001D9FFF7E1BF7047F838002038B501232A
:105EF000084C00252370656002F0A8FA02F0CEFA83
:105F00000549064802F0A4FB0223237085F311889B
:105F100038BD00BFA03B002040900008F8380020AA
:105F200000F080B9034A516853685B1A9842FBD865
:105F3000704700BF001000E08B604B630023CA6114
:105F400000F128020B6302230A618B84012388611C
:105F500081F8263001F11003C26A4A611360C362FE
:105F600001F12C030846CB6270470000D0E90131F3
:105F7000026841F8183CA1F19C033839CB600369F1
:105F800041F8243C436941F8203C034B41F8043C70
:105F9000C3680248FFF7D0BF1D040008F83800208E
:105FA00008B5FFF7E3FFBDE80840FFF741BF000079
:105FB00038B50E4BDC6804F12C05A062E06AA842FB
:105FC0000FD194F826303BB994F825309B0702BFD7
:105FD000D4E9043213605A600F20BDE83840FFF75F
:105FE00029BF0368E362FFF723FFE7E7F8380020E3
:105FF000302383F31188FFF7DBBF000008B50146AB
:10600000302383F311880820FFF724FF002383F354
:10601000118808BD054BDB6821B10360986203203D
:10602000FFF718BF4FF0FF30704700BFF83800206F
:1060300003682BB10022026018469962FFF7F8BE90
:1060400070470000064BDB6839B1426818605A603F
:10605000136043600420FFF7FDBE4FF0FF30704730
:10606000F83800200368984206D01A680260506031
:1060700018469962FFF7DCBE7047000038B5044649
:106080000D462068844200D138BD036823605C60FF
:106090008562FFF7CDFEF4E7036810B59C68A24265
:1060A0000CD85C688A600B604C602160596099680C
:1060B0008A1A9A604FF0FF33836010BD121B1B6871
:1060C000ECE700000A2938BF0A2170B504460D46E6
:1060D0000A26601902F0B6F902F0A2F9041BA542E3
:1060E00003D8751C04462E46F3E70A2E04D9012076
:1060F000BDE8704002F074BB70BD0000F8B5144BF1
:106100000D460A2A4FF00A07D96103F11001826097
:1061100038BF0A224160196914460160486018615D
:10612000A81802F081F902F07BF9431B0646A3424E
:1061300006D37C1C28192746354602F083F9F2E77E
:106140000A2F04D90120BDE8F84002F049BBF8BD90
:10615000F8380020F8B506460D4602F061F90F4AFE
:10616000134653F8107F9F4206D12A460146304617
:10617000BDE8F840FFF7C2BFD169BB68441A2C19CB
:1061800028BF2C46A34202D92946FFF79BFF22468F
:1061900031460348BDE8F840FFF77EBFF8380020DD
:1061A00008390020C0E90323002310B45DF8044B34
:1061B0004361FFF7CFBF000010B5194C2369984227
:1061C0000DD08168D0E9003213605A609A680A44A1
:1061D0009A60002303604FF0FF33A36110BD026893
:1061E000234643F8102F53600022026022699A422E
:1061F00003D1BDE8104002F01FB9936881680B44D9
:10620000936002F00DF92269E1699268441AA24292
:10621000E4D91144BDE81040091AFFF753BF00BF8D
:10622000F83800202DE9F047DFF8BC8008F11007AE
:106230002C4ED8F8105002F0F3F8D8F81C40AA6899
:10624000031B9A423ED814444FF00009D5E90032AE
:10625000C8F81C4013605A60C5F80090D8F8103098
:10626000B34201D102F0E8F889F31188D5E903318E
:1062700028469847302383F311886B69002BD8D0C8
:1062800002F0CEF86A69A0EB040982464A450DD2B5
:10629000022002F0A5FA0022D8F81030B34208D14B
:1062A00051462846BDE8F047FFF728BF121A22449E
:1062B000F2E712EB09092946384638BF4A46FFF78C
:1062C000EBFEB5E7D8F81030B34208D01444C8F854
:1062D0001C00211AA960BDE8F047FFF7F3BEBDE836
:1062E000F08700BF08390020F838002038B502F0E8
:1062F00097F8054AD2E90845031B181945F1000132
:10630000C2E9080138BD00BFF838002010B560B9F7
:10631000074804790368053C9B6818BF0124984727
:1063200008B144F00404204610BD0124FBE700BF7F
:10633000A0360020FFF7EABF2DE9F0478846174650
:106340009A460446B0B90D4E3579052D05D0032483
:106350000DE0013D15F0FF050ED032685346394679
:106360003046D2F814904246C8470028F1D1204662
:10637000BDE8F0870424FAE70124F8E7A0360020FE
:106380002DE9F047884617469A460446B0B90D4EA7
:106390003579052D05D003240DE0013D15F0FF05ED
:1063A0000ED03268534639463046D2F818904246ED
:1063B000C8470028F1D12046BDE8F0870424FAE759
:1063C0000124F8E7A036002037B50C46154670B911
:1063D00051B101290BD10748694603681B6A9847E8
:1063E00010B9019B04462B60204603B030BD042445
:1063F000FAE700BFA036002000207047FEE700004B
:10640000704700004FF0FF30704700004B6843605A
:106410008B688360CB68C3600B6943614B6903621F
:106420008B6943620B6803607047000008B53C4B02
:1064300040F2FF713B48D3F888200A43C3F8882014
:10644000D3F8882022F4FF6222F00702C3F88820E4
:10645000D3F88820D3F8E0200A43C3F8E020D3F82B
:1064600008210A43C3F808212F4AD3F808311146FE
:10647000FFF7CCFF00F5806002F11C01FFF7C6FFBB
:1064800000F5806002F13801FFF7C0FF00F5806081
:1064900002F15401FFF7BAFF00F5806002F17001CC
:1064A000FFF7B4FF00F5806002F18C01FFF7AEFF4B
:1064B00000F5806002F1A801FFF7A8FF00F58060F9
:1064C00002F1C401FFF7A2FF00F5806002F1E001D4
:1064D000FFF79CFF00F5806002F1FC01FFF796FFDB
:1064E00002F58C7100F58060FFF790FF01F070FC01
:1064F0000E4BD3F8902242F00102C3F89022D3F859
:10650000942242F00102C3F894220522C3F8982095
:106510004FF06052C3F89C20054AC3F8A02008BD84
:1065200000440258000002585490000800ED00E0BA
:106530001F00080308B501F037FDFFF7D7FC104B2B
:10654000D3F8DC2042F04002C3F8DC20D3F8042169
:1065500022F04002C3F80421D3F80431094B1A6831
:1065600042F008021A601A6842F004021A6000F051
:106570005DFD00F03DFBBDE8084000F0B5B800BF90
:10658000004402580018024801207047002070475C
:106590007047000002290CD0032904D001290748C4
:1065A00018BF00207047032A05D8054800EBC20039
:1065B0007047044870470020704700BF549200089D
:1065C000442200200892000870B59AB0054608469B
:1065D000144601A900F0C2F801A8FBF731FC431CE6
:1065E0000022C6B25B001046C5E9003423700323C5
:1065F000023404F8013C01ABD1B202348E4201D81E
:106600001AB070BD13F8011B013204F8010C04F834
:10661000021CF1E708B5302383F311880348FFF724
:106620009BF8002383F3118808BD00BFA83B00201E
:1066300090F8803003F01F02012A07D190F88120E2
:106640000B2A03D10023C0E91D3315E003F06003DA
:10665000202B08D1B0F884302BB990F88120212A62
:1066600003D81F2A04D8FFF759B8222AEBD0FAE73B
:10667000034A426707228267C3670120704700BF51
:106680003B22002007B5052917D8DFE801F01916CD
:1066900003191920302383F31188104A0121019036
:1066A000FFF702F9019802210D4AFFF7FDF80D48A6
:1066B000FFF71EF8002383F3118803B05DF804FB95
:1066C000302383F311880748FEF7E8FFF2E7302311
:1066D00083F311880348FEF7FFFFEBE7A89100085A
:1066E000CC910008A83B002038B50C4D0C4C2A4634
:1066F0000C4904F10800FFF767FF05F1CA0204F135
:1067000010000949FFF760FF05F5CA7204F118008F
:106710000649BDE83840FFF757BF00BF805400204E
:106720004422002088910008929100089D91000861
:1067300070B5044608460D46FBF782FBC6B22046FC
:10674000013403780BB9184670BD32462946FBF771
:1067500063FB0028F3D10120F6E700002DE9F047A4
:1067600005460C46FBF76CFB2A49C6B22846FFF7E4
:10677000DFFF08B10D36F6B227492846FFF7D8FFEC
:1067800008B11036F6B2632E0BD8DFF88880DFF838
:106790008890224FDFF890A02E7846B92670BDE889
:1067A000F08729462046BDE8F04702F0B5B8252E0F
:1067B0002CD1072241462846FBF72EFB60B9184B27
:1067C000224603F1140153F8040B8B4242F8040BE8
:1067D000F9D107351434DFE7082249462846FBF78C
:1067E0001BFB98B9A21C0F4B197802320909C95D2D
:1067F00002F8041C13F8011B01F00F015345C95D99
:1068000002F8031CF0D118340835C5E7013504F847
:10681000016BC1E7749200089D91000891920008F5
:106820007C92000800E8F11F0CE8F11FBFF34F8FC6
:10683000044B1A695107FCD1D3F810215207F8D143
:10684000704700BF0020005208B50D4B1B78ABB954
:10685000FFF7ECFF0B4BDA68D10704D50A4A5A6000
:1068600002F188325A60D3F80C21D20706D5064AC5
:10687000C3F8042102F18832C3F8042108BD00BF27
:10688000DE560020002000522301674508B5114B59
:106890001B78F3B9104B1A69510703D5DA6842F037
:1068A0004002DA60D3F81021520705D5D3F80C2145
:1068B00042F04002C3F80C21FFF7B8FF064BDA683C
:1068C00042F00102DA60D3F80C2142F00102C3F871
:1068D0000C2108BDDE560020002000520F289ABF70
:1068E00000F5806040040020704700004FF4003045
:1068F00070470000102070470F2808B50BD8FFF72D
:10690000EDFF00F500330268013204D10430834208
:10691000F9D1012008BD0020FCE700000F2838B5A0
:1069200005463FD8FFF782FF1F4CFFF78DFF4FF062
:10693000FF3307286361C4F814311DD82361FFF7C2
:1069400075FF030243F02403E360E36843F0800330
:10695000E36023695A07FCD42846FFF767FFFFF777
:10696000BDFF4FF4003100F09BFA2846FFF78EFF81
:10697000BDE83840FFF7C0BFC4F81031FFF756FF3D
:10698000A0F108031B0243F02403C4F80C31D4F82F
:106990000C3143F08003C4F80C31D4F810315B079C
:1069A000FBD4D9E7002038BD002000522DE9F84F74
:1069B00004460D46104644EA0203DE0602D00020DB
:1069C000BDE8F88F20F01F00DFF8D4B0DFF8D4A0C6
:1069D000FFF73AFF05EB0008454503D10120FFF71B
:1069E00055FFEDE720222946204601F05DFF10B952
:1069F00020342035F0E7234604F120021F68791C7B
:106A0000DDD104339342F9D104F178432048214E7B
:106A1000B3F5801F204B38BF184603F1F80332BF8F
:106A2000D946D1461E46FFF701FF0760A4EB050CCF
:106A3000336805F11C0143F0020333602B1FD9F8C2
:106A4000007017F00507FAD153F8042F8B424CF869
:106A50000320F4D1BFF34F8FFFF7E8FE4FF0FF3371
:106A60000360336823F002033360BFF34F8F0B4B97
:106A7000C3F85C42BFF34F8FBFF36F8F20222946CC
:106A8000204601F011FF0028B2D03846A7E700BF2A
:106A9000142100520C2000521420005200ED00E09E
:106AA000102000521021005210B5084C237828B154
:106AB0001BB9FFF7C9FE0123237010BD002BFCD0CA
:106AC0002070BDE81040FFF7E1BE00BFDE56002099
:106AD0002DE9F04F0D4685B0814658B111F00D06F5
:106AE00014BF2022082211F00803019304D0431E92
:106AF000034269D0002435E0002E37D009F11F0190
:106B000021F01F094FF00108314F05F00403DFF8B1
:106B1000CCA005EA080BBBF1000F32D07869C007A2
:106B20002FD408F101080C37B8F1060FF3D19EB944
:106B3000284D4946A819019201F0D2FC04460028CC
:106B400039D12036019AA02EF3D1494601F0C8FC74
:106B5000044600282FD1019A49461F4801F0C0FC85
:106B6000044660BB204605B0BDE8F08F0029C9D1BE
:106B700001462846029201F0B3FC0446D8B9029AB5
:106B8000C0E713B178694107CBD5AC0702D5786966
:106B90008007C6D5019911B178690107C1D5494669
:106BA0000AEB4810CDE9022301F09AFC0446DDE926
:106BB00002230028B5D04A460021204601E04A467B
:106BC0000021FBF745F9CDE70246002E96D199E763
:106BD000A492000820570020E05600200057002013
:106BE0000021FFF775BF00000121FFF771BF000012
:106BF00000231A4670B51A600433B3F5806FFAD1DA
:106C0000104D0124104E06EB441001342A6955F84A
:106C10000C1F01F051FC062CF5D137254FF4C05460
:106C20002046FFF7E1FF014628B122460748BDE8AC
:106C3000704001F041BCC4EBC404013D4FEAD404F0
:106C4000EED170BDA492000800570020E05600204D
:106C50000421FFF73DBF00004843FFF7C1BF00001C
:106C600008B101F0AFBC7047B0F5805F10B50446C5
:106C700007D8FFF7EDFF28B92046BDE81040FFF721
:106C8000AFBF002010BD0000FFF7EABF70B5AAB18A
:106C900040EA010313F01F030FD1094C0144A5681A
:106CA0006D0706D52568A84203D366683544A94216
:106CB00004D903330C34122BF1D10022104670BDDD
:106CC000A492000808B501F093FD034AD2E900320E
:106CD000C01842EB010108BDC0570020434BD3E967
:106CE00000232DE9F34113437CD0FFF7EBFF404A2B
:106CF00000230027F9F7A0FB06460D463D4A002376
:106D0000F9F79AFB0023144630462946394AF9F729
:106D100093FB4FF461613C23ADF80170B4FBF1F5D6
:106D2000B4FBF3F601FB154103FB16464624B1FB09
:106D3000F3F1314BF6B28DF8004098423CD84FF059
:106D4000640C4FF4C87EA30704F26C7225D1B2FB29
:106D5000FCF30CFB132313BBB2FBFEF30EFB13225D
:106D6000B2FA82F35B0903F26D18621C8045D2B25D
:106D700017D90FB18DF800400022204C4FF00C0CB9
:106D800017460CFB0343D4B2013213F804C0844508
:106D90000CD8A0EB0C000127F5E70023E3E7012363
:106DA000E1E7A0EB080014460127CCE70FB18DF80E
:106DB0000140431C8DF802309DF80100431C9DF8F2
:106DC00000005038400640EA43509DF8023040EA47
:106DD000034040EA560040EAC52040EA411002B0B4
:106DE000BDE8F0814FF40410F9E700BFC057002060
:106DF00040420F008051010090230B00EC920008EC
:106E00000244074BD2B210B5904200D110BD441CD1
:106E100000B253F8200041F8040BE0B2F4E700BFE1
:106E2000504000580E4B30B51C6F240405D41C6F25
:106E30001C671C6F44F400441C670A4C024423681E
:106E4000D2B243F480732360074B904200D130BD2F
:106E5000441C51F8045B00B243F82050E0B2F4E760
:106E600000440258004802585040005807B501221B
:106E700001A90020FFF7C4FF019803B05DF804FBEF
:106E800013B50446FFF7F2FFA04205D0012201A985
:106E900000200194FFF7C6FF02B010BD704700004C
:106EA0000144BFF34F8F064B884204D3BFF34F8F8B
:106EB000BFF36F8F7047C3F85C022030F4E700BF68
:106EC00000ED00E00144BFF34F8F064B884204D32E
:106ED000BFF34F8FBFF36F8F7047C3F8700220303E
:106EE000F4E700BF00ED00E070B5054616460C461D
:106EF00001201021FFF7B0FE286046733CB1204608
:106F000036B1FFF7A5FE2B68186000B19C6070BD1C
:106F1000FFF76AFEF7E70000F8B50F46154604468E
:106F200048B905F11F010126386821F01F01FFF75C
:106F3000B7FF3046F8BD427B29463868FFF7A6FE0A
:106F400006460028EDD13B686360A368AB4210D2CF
:106F500013B12068FFF784FE637B28462BB1FFF74F
:106F600077FE206020B9A060E3E7FFF73DFEF8E779
:106F7000A560206805F11F01012621F01F0138607E
:106F8000FFF78EFF2673D4E710B5044640B10068C2
:106F9000884205D1606808B1FAF734FF00232373F3
:106FA00010BD0000F8B50F461446054648B904F177
:106FB0001F010126386821F01F01FFF783FF3046CB
:106FC000F8BD427B21463868FFF760FE0646002880
:106FD000EDD1AB68A34210D213B12868FFF740FE91
:106FE0006B7B20462BB1FFF733FE286020B9A860E9
:106FF000E5E7FFF7F9FDF8E7AC60396819B122461B
:107000002868FAF7FFFE286804F11F01012621F025
:107010001F013860FFF756FF2E73D0E720B10368D9
:107020008B4204BF0023037370470000034B1A68B0
:107030001AB9034AD2F8D0241A607047C857002002
:107040000040025808B5FFF7F1FF024B1868C0F383
:10705000806008BDC8570020EFF3098305496833F5
:107060004A6B22F001024A6383F30988002383F309
:107070001188704700EF00E0302080F3118862B67D
:107080000D4B0E4AD96821F4E0610904090C0A434A
:107090000B49DA60D3F8FC2042F08072C3F8FC2080
:1070A000084AC2F8B01F116841F0010111602022A6
:1070B000DA7783F82200704700ED00E00003FA055C
:1070C00055CEACC5001000E0302310B583F3118815
:1070D0000E4B5B6813F4006314D0F1EE103AEFF33B
:1070E00009844FF08073683CE361094BDB6B2366D6
:1070F00084F30988FEF7CCFE10B1064BA36110BDE6
:10710000054BFBE783F31188F9E700BF00ED00E0D2
:1071100000EF00E02F0400083204000870B5BFF350
:107120004F8FBFF36F8F1A4A0021C2F85012BFF37E
:107130004F8FBFF36F8F536943F400335361BFF335
:107140004F8FBFF36F8FC2F88410BFF34F8FD2F809
:10715000803043F6E074C3F3C900C3F34E335B01E0
:1071600003EA0406014646EA81750139C2F8605215
:10717000F9D2203B13F1200FF2D1BFF34F8F5369A7
:1071800043F480335361BFF34F8FBFF36F8F70BDF4
:1071900000ED00E0FEE70000214B2248224A70B5D6
:1071A000904237D3214BC11EDA1C121A22F003027F
:1071B0008B4238BF00220021FAF74AFE1C4A002306
:1071C000C2F88430BFF34F8FD2F8803043F6E074BA
:1071D000C3F3C900C3F34E335B0103EA040601465F
:1071E00046EA81750139C2F86C52F9D2203B13F19D
:1071F000200FF2D1BFF34F8FBFF36F8FBFF34F8FCD
:10720000BFF36F8F0023C2F85032BFF34F8FBFF32D
:107210006F8F70BD53F8041B40F8041BC0E700BF1C
:10722000E4930008445900204459002044590020A8
:1072300000ED00E0074BD3F8D81021EA0001C3F8B5
:10724000D810D3F8002122EA0002C3F80021D3F8B5
:10725000003170470044025870B5D0E92443002241
:107260004FF0FF359E6804EB42135101D3F800093B
:10727000002805DAD3F8000940F08040C3F800097F
:10728000D3F8000B002805DAD3F8000B40F080405B
:10729000C3F8000B013263189642C3F80859C3F8CB
:1072A000085BE0D24FF00113C4F81C3870BD000039
:1072B000890141F02001016103699B06FCD4122081
:1072C000FEF730BE10B50A4C2046FEF7CBFA094B4C
:1072D000C4F89030084BC4F89430084C2046FEF7B0
:1072E000C1FA074BC4F89030064BC4F8943010BD77
:1072F000CC57002000000840289300086858002060
:10730000000004403493000870B503780546012B53
:107310005CD1434BD0F89040984258D1414B0E215C
:107320006520D3F8D82042F00062C3F8D820D3F803
:10733000002142F00062C3F80021D3F80021D3F805
:10734000802042F00062C3F88020D3F8802022F031
:107350000062C3F88020D3F88030FDF78DFE324BF9
:10736000E360324BC4F800380023D5F89060C4F8CD
:10737000003EC02323604FF40413A3633369002B42
:10738000FCDA01230C203361FEF7CCFD3369DB0707
:10739000FCD41220FEF7C6FD3369002BFCDA002670
:1073A0002846A660FFF758FF6B68C4F81068DB68D2
:1073B000C4F81468C4F81C6883BB1D4BA3614FF06C
:1073C000FF336361A36843F00103A36070BD194BF1
:1073D0009842C9D1134B4FF08060D3F8D82042F0C7
:1073E0000072C3F8D820D3F8002142F00072C3F82D
:1073F0000021D3F80021D3F8802042F00072C3F8B6
:107400008020D3F8802022F00072C3F88020D3F8C7
:107410008030FFF70FFF0E214D209EE7064BCDE792
:10742000CC570020004402584014004003002002C2
:10743000003C30C068580020083C30C0F8B5D0F897
:107440009040054600214FF000662046FFF730FFD0
:10745000D5F8941000234FF001128F684FF0FF30E1
:10746000C4F83438C4F81C2804EB431201339F429B
:10747000C2F80069C2F8006BC2F80809C2F8080B2C
:10748000F2D20B68D5F89020C5F8983063621023CB
:107490001361166916F01006FBD11220FEF742FDAB
:1074A000D4F8003823F4FE63C4F80038A36943F429
:1074B000402343F01003A3610923C4F81038C4F833
:1074C00014380B4BEB604FF0C043C4F8103B094B32
:1074D000C4F8003BC4F81069C4F80039D5F89830F6
:1074E00003F1100243F48013C5F89820A362F8BD9D
:1074F0000493000840800010D0F8902090F88A1083
:10750000D2F8003823F4FE6343EA0113C2F80038CE
:10751000704700002DE9F84300EB8103D0F890504C
:107520000C468046DA680FFA81F94801166806F0C1
:107530000306731E022B05EB41134FF0000194BFAD
:10754000B604384EC3F8101B4FF0010104F11003CC
:1075500098BF06F1805601FA03F3916998BF06F5CA
:10756000004600293AD0578A04F1580137434901AF
:107570006F50D5F81C180B430021C5F81C382B1888
:107580000127C3F81019A7405369611E9BB3138AE2
:10759000928B9B08012A88BF5343D8F898209818EB
:1075A00042EA034301F140022146C8F89800284608
:1075B00005EB82025360FFF77BFE08EB8900C3688E
:1075C0001B8A43EA845348341E4364012E51D5F884
:1075D0001C381F43C5F81C78BDE8F88305EB491734
:1075E000D7F8001B21F40041C7F8001BD5F81C1880
:1075F00021EA0303C0E704F13F030B4A2846214672
:1076000005EB83035A60FFF753FE05EB4910D0F8F2
:10761000003923F40043C0F80039D5F81C3823EAB8
:107620000707D7E70080001000040002D0F894207C
:107630001268C0F89820FFF70FBE00005831D0F84C
:10764000903049015B5813F4004004D013F4001F3C
:107650000CBF0220012070474831D0F8903049011A
:107660005B5813F4004004D013F4001F0CBF022039
:107670000120704700EB8101CB68196A0B68136029
:107680004B6853607047000000EB810330B5DD6844
:10769000AA691368D36019B9402B84BF40231360D3
:1076A0006B8A1468D0F890201C4402EB4110013C16
:1076B00009B2B4FBF3F46343033323F0030343EA57
:1076C000C44343F0C043C0F8103B2B6803F00303EE
:1076D000012B0ED1D2F8083802EB411013F4807F51
:1076E000D0F8003B14BF43F0805343F00053C0F880
:1076F000003B02EB4112D2F8003B43F00443C2F8D6
:10770000003B30BD2DE9F041D0F8906005460C46B5
:1077100006EB4113D3F8087B3A07C3F8087B08D57A
:10772000D6F814381B0704D500EB8103DB685B68CF
:107730009847FA071FD5D6F81438DB071BD505EB99
:107740008403D968CCB98B69488A5A68B2FBF0F6D1
:1077500000FB16228AB91868DA6890420DD2121A14
:10776000C3E90024302383F3118821462846FFF71C
:107770008BFF84F31188BDE8F081012303FA04F242
:107780006B8923EA02036B81CB68002BF3D021467F
:107790002846BDE8F041184700EB81034A0170B567
:1077A000DD68D0F890306C692668E66056BB1A44F4
:1077B0004FF40020C2F810092A6802F00302012ADF
:1077C0000AB20ED1D3F8080803EB421410F4807FFC
:1077D000D4F8000914BF40F0805040F00050C4F8C5
:1077E000000903EB4212D2F8000940F00440C2F84D
:1077F00000090122D3F8340802FA01F10143C3F869
:10780000341870BD19B9402E84BF40202060206814
:107810001A442E8A8419013CB4FBF6F440EAC440B1
:1078200040F00050C6E700002DE9F843D0F8906022
:1078300005460C464F0106EB4113D3F8088918F0B2
:10784000010FC3F808891CD0D6F81038DB0718D50B
:1078500000EB8103D3F80CC0DCF81430D3F800E05F
:10786000DA68964530D2A2EB0E024FF000091A609A
:10787000C3F80490302383F31188FFF78DFF89F359
:10788000118818F0800F1DD0D6F834380126A64094
:10789000334217D005EB84030134D5F89050D3F868
:1078A0000CC0E4B22F44DCF8142005EB0434D2F809
:1078B00000E05168714514D3D5F8343823EA060640
:1078C000C5F83468BDE8F883012303FA01F203899F
:1078D00023EA02030381DCF80830002BD1D098475B
:1078E000CFE7AEEB0103BCF81000834228BF03468C
:1078F000D7F8180980B2B3EB800FE3D89068A0F1F5
:10790000040959F8048FC4F80080A0EB09089844D2
:10791000B8F1040FF5D818440B4490605360C8E7E1
:107920002DE9F84FD0F8905004466E69AB691E40BF
:1079300016F480586E6103D0BDE8F84FFEF702B828
:10794000002E12DAD5F8003E9B0705D0D5F8003E90
:1079500023F00303C5F8003ED5F80438204623F091
:107960000103C5F80438FEF71BF8370505D5204696
:10797000FFF772FC2046FEF701F8B0040CD5D5F8ED
:10798000083813F0060FEB6823F470530CBF43F470
:10799000105343F4A053EB6031071BD56368DB68D9
:1079A0001BB9AB6923F00803AB612378052B0CD11D
:1079B000D5F8003E9A0705D0D5F8003E23F0030322
:1079C000C5F8003E2046FDF7EBFF6368DB680BB1AE
:1079D00020469847F30200F1BA80B70226D5D4F8C2
:1079E000909000274FF0010A09EB4712D2F8003BB4
:1079F00003F44023B3F5802F11D1D2F8003B002BC4
:107A00000DDA62890AFA07F322EA0303638104EBC1
:107A10008703DB68DB6813B1394620469847013796
:107A2000D4F89430FFB29B689F42DDD9F00619D597
:107A3000D4F89000026AC2F30A1702F00F0302F4AE
:107A4000F012B2F5802F00F0CA80B2F5402F09D1B4
:107A500004EB8303002200F58050DB681B6A974229
:107A600040F0B0803003D5F8185835D5E90303D578
:107A700000212046FFF746FEAA0303D50121204638
:107A8000FFF740FE6B0303D502212046FFF73AFEC5
:107A90002F0303D503212046FFF734FEE80203D568
:107AA00004212046FFF72EFEA90203D5052120461A
:107AB000FFF728FE6A0203D506212046FFF722FEC3
:107AC0002B0203D507212046FFF71CFEEF0103D54B
:107AD00008212046FFF716FE700340F1A780E90752
:107AE00003D500212046FFF79FFEAA0703D50121F9
:107AF0002046FFF799FE6B0703D502212046FFF7CA
:107B000093FE2F0703D503212046FFF78DFEEE06D7
:107B100003D504212046FFF787FEA80603D50521DB
:107B20002046FFF781FE690603D506212046FFF7B0
:107B30007BFE2A0603D507212046FFF775FEEB05DD
:107B400074D520460821BDE8F84FFFF76DBED4F884
:107B500090904FF0000B4FF0010AD4F894305FFA88
:107B60008BF79B689F423FF638AF09EB4713D3F87A
:107B7000002902F44022B2F5802F20D1D3F8002949
:107B8000002A1CDAD3F8002942F09042C3F80029F9
:107B9000D3F80029002AFBDB3946D4F89000FFF720
:107BA00087FB22890AFA07F322EA0303238104EB05
:107BB0008703DB689B6813B13946204698470BF171
:107BC000010BCAE7910701D1D0F80080072A02F122
:107BD00001029CBF03F8018B4FEA18283FE704EB32
:107BE000830300F58050DA68D2F818C0DCF808206A
:107BF000DCE9001CA1EB0C0C00218F4208D1DB68F2
:107C00009B699A683A449A605A683A445A6029E7EC
:107C100011F0030F01D1D0F800808C4501F1010172
:107C200084BF02F8018B4FEA1828E6E7BDE8F88F19
:107C300008B50348FFF774FEBDE80840FFF744BAF3
:107C4000CC57002008B50348FFF76AFEBDE808409E
:107C5000FFF73ABA68580020D0F8903003EB411192
:107C6000D1F8003B43F40013C1F8003B704700001B
:107C7000D0F8903003EB4111D1F8003943F40013F0
:107C8000C1F8003970470000D0F8903003EB411183
:107C9000D1F8003B23F40013C1F8003B704700000B
:107CA000D0F8903003EB4111D1F8003923F40013E0
:107CB000C1F8003970470000064BD3F8DC200243BE
:107CC000C3F8DC20D3F804211043C3F80401D3F82F
:107CD000043170470044025808B53C4B4FF0FF3167
:107CE000D3F8802062F00042C3F88020D3F88020CF
:107CF00002F00042C3F88020D3F88020D3F884201B
:107D0000C3F88410D3F884200022C3F88420D3F869
:107D10008400D86F40F0FF4040F4FF0040F4DF40A3
:107D200040F07F00D867D86F20F0FF4020F4FF00BC
:107D300020F4DF4020F07F00D867D86FD3F88800A8
:107D40006FEA40506FEA5050C3F88800D3F88800BB
:107D5000C0F30A00C3F88800D3F88800D3F8900075
:107D6000C3F89010D3F89000C3F89020D3F8900097
:107D7000D3F89400C3F89410D3F89400C3F8942077
:107D8000D3F89400D3F89800C3F89810D3F898006B
:107D9000C3F89820D3F89800D3F88C00C3F88C105F
:107DA000D3F88C00C3F88C20D3F88C00D3F89C0057
:107DB000C3F89C10D3F89C10C3F89C20D3F89C30D7
:107DC000FCF784FDBDE8084000F0DEB8004402582E
:107DD00008B50122534BC3F80821534BD3F8F420C4
:107DE00042F00202C3F8F420D3F81C2142F0020250
:107DF000C3F81C210222D3F81C314C4BDA605A68BC
:107E00009104FCD54A4A1A6001229A60494ADA6014
:107E100000221A614FF440429A61444B9A699204DD
:107E2000FCD51A6842F480721A603F4B1A6F12F444
:107E3000407F04D04FF480321A6700221A671A6814
:107E400042F001021A60384B1A685007FCD5002234
:107E50001A611A6912F03802FBD1012119604FF042
:107E6000804159605A67344ADA62344A1A611A68A2
:107E700042F480321A602C4B1A689103FCD51A68C0
:107E800042F480521A601A689204FCD52C4A2D499B
:107E90009A6200225A63196301F57C01DA6301F2E8
:107EA000E71199635A64284A1A64284ADA621A6800
:107EB00042F0A8521A601C4B1A6802F02852B2F124
:107EC000285FF9D148229A614FF48862DA61402232
:107ED0001A621F4ADA641F4A1A651F4A5A651F4A06
:107EE0009A6532231E4A1360136803F00F03022BB6
:107EF000FAD10D4A136943F003031361136903F0C8
:107F00003803182BFAD14FF00050FFF7D5FE4FF091
:107F10008040FFF7D1FE4FF00040BDE80840FFF77A
:107F2000CBBE00BF008000510044025800480258F8
:107F300000C000F0020000010000FF01008890086E
:107F40002220400063020901470E0508DD0BBF0136
:107F500020000020000001100910E00000010110C5
:107F60000020005208B50348FDF778F8BDE8084046
:107F7000FFF7AAB8A036002008B500F07FFCBDE8E6
:107F80000840FFF7A1B8000008B509217A20FDF7E5
:107F900073F809213120FDF76FF807211C20BDE897
:107FA0000840FDF769B8000008B5FFF795FE00F03E
:107FB0003BFCFDF785FAFDF753FCFDF725FBFEF7CB
:107FC000E7FABDE8084000F029BA000030B50433F4
:107FD000039C0172002104FB0325C160C0E9065324
:107FE000049B0363059BC0E90000C0E90422C0E9CB
:107FF0000842C0E90A11436330BD00000022416A13
:10800000C260C0E90411C0E90A226FF00101FEF765
:1080100035B80000D0E90432934201D1C2680AB9F0
:10802000181D704700207047036919600021C2685D
:108030000132C260C269134482699342036124BF62
:10804000436A0361FEF70EB838B504460D46E3688F
:108050003BB162690020131D1268A3621344E362FE
:1080600007E0237A33B929462046FDF7EBFF0028C5
:10807000EDDA38BD6FF00100FBE70000C368C269AC
:10808000013BC3604369134482699342436124BF47
:10809000436A436100238362036B03B1184770474F
:1080A00070B53023044683F31188866A3EB9FFF722
:1080B000CBFF054618B186F31188284670BDA36A28
:1080C000E26A13F8015B9342A36202D32046FFF7F2
:1080D000D5FF002383F31188EFE700002DE9F84F67
:1080E00004460E46174698464FF0300989F311882A
:1080F0000025AA46D4F828B0BBF1000F09D14146AB
:108100002046FFF7A1FF20B18BF311882846BDE878
:10811000F88FD4E90A12A7EB050B521A934528BF32
:108120009346BBF1400F1BD9334601F1400251F891
:10813000040B914243F8040BF9D1A36A4036403551
:108140004033A362D4E90A239A4202D32046FFF7C0
:1081500095FF8AF31188BD42D8D289F31188C9E707
:1081600030465A46F9F74EFEA36A5E445D445B44CE
:10817000A362E7E710B5029C0433017203FB0421FC
:10818000C460C0E906130023C0E90A33039B0363FC
:10819000049BC0E90000C0E90422C0E9084243632F
:1081A00010BD0000026A6FF00101C260426AC0E9BE
:1081B00004220022C0E90A22FDF760BFD0E90423AF
:1081C0009A4201D1C26822B9184650F8043B0B60AC
:1081D000704700231846FAE7C3680021C2690133DB
:1081E000C3604369134482699342436124BF436A75
:1081F0004361FDF737BF000038B504460D46E3681C
:108200003BB1236900201A1DA262E2691344E362B4
:1082100007E0237A33B929462046FDF713FF0028EB
:10822000EDDA38BD6FF00100FBE70000036919606B
:10823000C268013AC260C269134482699342036111
:1082400024BF436A036100238362036B03B11847B1
:108250007047000070B530230D460446114683F385
:108260001188866A2EB9FFF7C7FF10B186F311880F
:1082700070BDA36A1D70A36AE26A01339342A362D0
:1082800004D3E16920460439FFF7D0FF002080F3D2
:108290001188EDE72DE9F84F04460D4690469946C2
:1082A0004FF0300A8AF311880026B346A76A4FB907
:1082B00049462046FFF7A0FF20B187F311883046DA
:1082C000BDE8F88FD4E90A073A1AA8EB06079742E7
:1082D00028BF1746402F1BD905F1400355F8042B42
:1082E0009D4240F8042BF9D1A36A40364033A36283
:1082F000D4E90A239A4204D3E16920460439FFF7FE
:1083000095FF8BF311884645D9D28AF31188CDE7C2
:1083100029463A46F9F776FDA36A3D443E443B447C
:10832000A362E5E7D0E904239A4217D1C3689BB161
:10833000836A8BB1043B9B1A0ED01360C368013B68
:10834000C360C3691A4483699A42026124BF436AC5
:108350000361002383620123184670470023FBE773
:1083600001F01F03F0B502F01F0456095A1C012347
:10837000B6EB511F50F8265003FA02F34FEA51179B
:1083800003F1FF333DBF50F82720C4F12000134014
:1083900003EA05003BBF03FA00F225FA04F0E040CF
:1083A0001043F0BD70B57E227F210546FFF7D8FF50
:1083B00018B1012819D0002070BD3E22492128465D
:1083C000FFF7CEFF2F22044631212846FFF7C8FFD2
:1083D000064601345022023653212846B440FFF7A6
:1083E000BFFF093804FA00F0E6E7302245212846AD
:1083F000FFF7B6FF01308002DEE7000090F8D630CC
:1084000090F8D7201B0403EB026390F8D42090F877
:10841000D500134403EB00207047000000F006BABB
:108420004FF08043586A70474FF0804300225863F2
:108430001A610222DA6070474FF080430022DA604E
:10844000704700004FF0804358637047024B034A67
:108450001A60034A5A6070471C590020485900208E
:1084600000000220074B494210B55C68201A084002
:108470001968821A8A4203D3A24201D85A6010BDF9
:108480000020FCE71C59002008B5302383F3118835
:10849000FFF7E8FF002383F3118808BD0448054B6C
:1084A00003600023C0E901330C3000F017B900BFAE
:1084B0002459002089840008CB1D083A23F00703C3
:1084C000591A521A10B4D2080024C0E9004384603B
:1084D0000C301C605A605DF8044B00F0FFB80000DF
:1084E0002DE9F74F364FCD1D8846002818BF0746A7
:1084F000082A4FEAD50538BF082207F10C003C1DB9
:108500009146019000F02CF9019809F10701C9F199
:10851000000E2246246864B900F02CF93B68CBB306
:1085200008224946E8009847044698B340E9027893
:1085300030E004EB010CD4F804A00CEA0E0C0AF1B4
:108540000106ACF1080304EBC6069E42E1D9A6EB96
:108550000C0CB5EBEC0F4FEAEC0BDAD89C421DD2B9
:1085600004F10802AB45A3EB02024FEAE2026260AB
:1085700009D9691CED4303EBC1025D4455602568D0
:1085800043F8315022601C46C3F8048044F8087B4D
:1085900000F0F0F8204603B0BDE8F08FAA4521684E
:1085A00002D111602346EEE7013504EBC50344F820
:1085B000351003F10801761AF6105E601360F1E7DA
:1085C0002459002073B50446A0F1080550F8080CA2
:1085D00054F8043C061D0C3007330190DB0844F8C6
:1085E000043C00F0BDF8334601989E421A6801D061
:1085F000AB4228D20AB1954225D244F8082C54F84F
:10860000042C1D60013254F8081C05EBC206B1426F
:1086100006D14E68324444F8042C0A6844F8082C09
:108620005E68711C03EBC1018D4207D154F8042C24
:10863000013232445A6054F8082C1A6002B0BDE886
:10864000704000F097B81346CFE70000FEE7000047
:1086500070B51E4B0025044686B058600E46056373
:108660008163FEF709FD04F12803A5606563C4E991
:108670000A3304F11003C4E904334FF0FF33C4E9B3
:108680000044C4E90635FFF7CBFE2B46024604F151
:108690003C012046C4E9082380230D4A6567FDF7A5
:1086A0004BFC7368E0600B4A03620123009280F880
:1086B00024306846F26801923269CDE90223064B04
:1086C000CDE90435FDF76CFC06B070BDA03B002081
:1086D00048930008409300084D8600080023C0E935
:1086E000000083600361704770B51C4B05468468C9
:1086F000DE685CB3B44213D103690133036170BD1A
:10870000A36094F8243083B1062B15D1A06A2146CA
:10871000D4E9003213605A60FDF77AFBA36A9C68C3
:10872000B368A2689A42EBD306E0D4E9003220464F
:1087300013605A60FDF77CFB28463146FDF768FB65
:10874000B5620620BDE87040FDF774BB0369866022
:1087500001330361336BC3603063D0E7F838002026
:1087600008B5302383F31188FFF7BEFF002383F39E
:10877000118808BD194BD96883688B4210B520D188
:10878000302383F311880269013A0261B2B90468A7
:10879000C368A0420B631ED04A6B9BB901238A6059
:1087A000036103681A68026050601A6B8360C260DC
:1087B00018631846FDF73CFBFDF78CFB002383F3A1
:1087C000118810BD1C68A34203D0A468A24238BF20
:1087D0002246DB68E1E78260F0E700BFF83800205E
:1087E000024A536B18435063704700BFF8380020AB
:1087F00038B5EFF311859DB9EFF30584C4F3080490
:10880000302334B183F31188FDF770FD85F31188AF
:1088100038BD83F31188FDF769FD84F3118838BDF5
:10882000BDE83840FDF762BD70470000114BD3F83A
:10883000E82042F00102C3F8E820D3F8102142F00A
:108840000102C3F810210C4AD3F81031D36B43F066
:108850000103D3634FF08043C7229A624FF0FF3287
:10886000DA6200229A615A63DA605A6001225A6120
:108870001A607047004402580010005C4FF08042BC
:1088800008B51169D3680B40D9B29B076FEA0101A3
:10889000116107D5302383F31188FDF741FB0023D5
:1088A00083F3118808BD000010B5013902449042DD
:1088B00001D1002005E0037811F8014FA34201D057
:1088C000181B10BD0130F2E7884210B501EB02041D
:1088D00002D98442234607D8431EA14208D011F88A
:1088E000012B03F8012FF8E7024401468A4200D128
:1088F00010BD13F8014D02F8014DF7E7C9B2034668
:1089000010F8012B1AB18A42F9D118467047002994
:1089100018BF0023F9E70000034611F8012B03F804
:10892000012B002AF9D1704710B50139034632B145
:1089300011F8014F03F8014B013A002CF7D11A440A
:108940000021934200D110BD03F8011BF9E700009C
:108950003630376239646664656631656432303456
:10896000000000001210000012110000121300009D
:108970004D4435002D2D0A002F6172647570696CAD
:108980006F742E6162696E002F6172647570696C1C
:108990006F742D7665726966792E6162696E002F3B
:1089A0006172647570696C6F742D666C6173682E8A
:1089B0006162696E002F6172647570696C6F742DED
:1089C000666C61736865642E6162696E0000000008
:1089D0000000000000000000150F0008B10F0008A3
:1089E00061110008E90F0008A90F0008000000004D
:1089F00000000000110F0008BD0F000899110008C9
:108A00000D0F0008190F000853544D333248373FFB
:108A10003F3F0053544D3332483733782F37327845
:108A20000053544D3332483734332F3735332F37D3
:108A30003530000001105A00031059000120580081
:108A4000032056002F00000053756363657373663F
:108A5000756C6C79206D6F756E746564205344433A
:108A60006172642028736C6F77646F776E3D257533
:108A7000290A0000EB7690455846415420202000FA
:108A80004641543332202020000000002A3A3C3E68
:108A90007C223F7F002B2C3B3D5B5D0043554541D5
:108AA0004141414345454549494941414592924FDC
:108AB0004F4F5555594F554F9C4F9E9F41494F55CC
:108AC000A5A5A6A7A8A9AAABACADAEAFB0B1B2B3ED
:108AD000B4414141B8B9BABBBCBDBEBFC0C1C2C33D
:108AE000C4C54141C8C9CACBCCCDCECFD1D14545F3
:108AF0004549494949D9DADBDCDD49DF4FE14F4FD0
:108B00004F4FE6E8E85555555959EEEFF0F1F2F3BD
:108B1000F4F5F6F7F8F9FAFBFCFDFEFF0103050793
:108B2000090E10121416181C1E00000061001A0312
:108B3000E0001703F8000703FF00010078010001BF
:108B4000300132010601390110014A012E0179017B
:108B5000060180014D0043028101820182018401EE
:108B6000840186018701870189018A018B018B01BC
:108B70008D018E018F01900191019101930194016A
:108B8000F60196019701980198013D029B019C0115
:108B90009D0120029F01A001A001A201A201A40148
:108BA000A401A601A701A701A901AA01AB01AC017B
:108BB000AC01AE01AF01AF01B101B201B301B3012C
:108BC000B501B501B701B801B801BA01BB01BC01DB
:108BD000BC01BE01F701C001C101C201C301C40152
:108BE000C501C401C701C801C701CA01CB01CA013F
:108BF000CD011001DD0101008E01DE011201F30142
:108C00000300F101F401F401F8012801220212012C
:108C10003A020900652C3B023B023D02662C3F02F2
:108C200040024102410246020A0153024000810112
:108C30008601550289018A0158028F015A0290016A
:108C40005C025D025E025F029301610262029401B6
:108C50006402650266026702970196016A02622C4D
:108C60006C026D026E029C01700271029D01730222
:108C700074029F0176027702780279027A027B02FF
:108C80007C02642C7E027F02A60181028202A9017D
:108C90008402850286028702AE014402B101B2015C
:108CA00045028D028E028F0290029102B7017B0372
:108CB0000300FD03FE03FF03AC03040086038803E7
:108CC00089038A03B1031103C2030200A303A303B0
:108CD000C4030803CC0303008C038E038F03D80363
:108CE0001801F2030A00F903F303F403F503F60392
:108CF000F703F703F903FA03FA03300420035004DF
:108D00001007600422018A043601C1040E01CF0459
:108D10000100C004D00444016105260400000000E5
:108D20007D1D0100632C001E9601A01E5A01001F2C
:108D30000806101F0606201F0806301F0806401FE1
:108D40000606511F0700591F521F5B1F541F5D1F4E
:108D5000561F5F1F601F0806701F0E00BA1FBB1F43
:108D6000C81FC91FCA1FCB1FDA1FDB1FF81FF91F3F
:108D7000EA1FEB1FFA1FFB1F801F0806901F080643
:108D8000A01F0806B01F0400B81FB91FB21FBC1FE8
:108D9000CC1F0100C31FD01F0206E01F0206E51F03
:108DA0000100EC1FF31F0100FC1F4E2101003221C6
:108DB00070211002842101008321D0241A05302C57
:108DC0002F04602C0201672C0601752C0201802CF7
:108DD0006401002D260841FF1A030000C700FC00B3
:108DE000E900E200E400E000E500E700EA00EB0053
:108DF000E800EF00EE00EC00C400C500C900E6008A
:108E0000C600F400F600F200FB00F900FF00D600F7
:108E1000DC00F800A300D800D7009201E100ED00CB
:108E2000F300FA00F100D100AA00BA00BF00AE00C2
:108E3000AC00BD00BC00A100AB00BB009125922599
:108E4000932502252425C100C200C000A900632586
:108E5000512557255D25A200A50010251425342590
:108E60002C251C2500253C25E300C3005A2554254C
:108E700069256625602550256C25A400F000D000EA
:108E8000CA00CB00C8003101CD00CE00CF001825AC
:108E90000C2588258425A600CC008025D300DF0082
:108EA000D400D200F500D500B500FE00DE00DA00E7
:108EB000DB00D900FD00DD00AF00B400AD00B10063
:108EC0001720BE00B600A700F700B800B000A80049
:108ED000B700B900B300B200A025A0001000024006
:108EE000080002400008024000000B002800024079
:108EF000080002400408024006010C004000024045
:108F0000080002400808024010020D00580002400C
:108F1000080002400C08024016030E0070000240D8
:108F20000C0002401008024000040F0088000240BC
:108F30000C0002401408024006051000A000024088
:108F40000C0002401808024010061100B800024050
:108F50000C0002401C08024016072F0010040240BB
:108F6000080402402008024000083800280402409B
:108F70000804024024080240060939004004024067
:108F80000804024028080240100A3A00580402402F
:108F9000080402402C080240160B3B0070040240FB
:108FA0000C04024030080240000C3C0088040240DF
:108FB0000C04024034080240060D4400A0040240A4
:108FC0000C04024038080240100E4500B80402406C
:108FD0000C0402403C080240160F4600010000004D
:108FE0000000000000000000896500088D65000891
:108FF000555100088D540008E9500008115100082F
:1090000039510008D15000080000000085550008C3
:1090100071550008AD55000899550008A555000880
:10902000915500087D55000869550008B95500089C
:10903000000000000100000000000000633000009C
:109040003C90000800000000000000007039002083
:10905000A03B00200000800200000000AAAAAAAAEB
:1090600000000000FFFF00000000000000A00A0058
:109070000100004000000000AAAAAAAA0100000006
:10908000FFFF000000000000000000000000AA0236
:1090900000000000AAAAAAAA00005500FFFF0000D5
:1090A00000000000CCCC0C002000000000000000FC
:1090B000AAAAAAAA10000000FFFF0000000C0000EE
:1090C000000000001000000000000000AAAAAAAAE8
:1090D00000000000FBFF0000000000000000000096
:1090E0000000000000000000AAAAAAAA00000000D8
:1090F000FFFF000000000000000000000000000072
:1091000000000000AAAAAAAA00000000FFFF0000B9
:10911000000000000000000000000000000000004F
:10912000AAAAAAAA00000000FFFF00000000000099
:10913000000000000000000000000000AAAAAAAA87
:1091400000000000FFFF0000000000000000000021
:109150000000000000000000AAAAAAAA0000000067
:10916000FFFF000000000000000000000000000001
:1091700000000000AAAAAAAA00000000FFFF000049
:1091800000000000000000004172647550696C6FBF
:10919000740025424F415244252D424C0025534531
:1091A0005249414C25000000020000000000000070
:1091B000A5570008155800084000400050540020F2
:1091C00060540020020000000000000003000000C6
:1091D000000000005D5800080000000010000000C2
:1091E000705400200000000001000000000000009A
:1091F000CC57002001010200856600089565000833
:10920000316600081566000843000000109200084F
:1092100009024300020100C03209040000010202F9
:1092200001000524001001052401000104240202AC
:109230000524060001070582030800FF0904010058
:10924000020A000000070501024000000705810234
:1092500040000000120000005C92000812011001A2
:109260000200004009124157000201020301000000
:109270000403090425424F41524425004165726FA1
:10928000436F6769746F2D48374469676974616C0F
:109290000030313233343536373839414243444572
:1092A0004600000000000020000002000200000054
:1092B000000000300000040008000000000000244E
:1092C00000000800040000000004000000FC000092
:1092D00002000000000004300080000008000000D0
:1092E0000000003800000100010000001F1C1F1ECC
:1092F0001F1E1F1F1E1F1E1F1F1D1F1E1F1E1F1F85
:109300001E1F1E1F00000000B9590008715C0008F4
:109310001D5D000840004000045900200459002051
:1093200001000000145900208000000040010000EE
:10933000080000000001000000100000080000000C
:1093400069646C65000000006D61696E002C043872
:10935000040438080C10141C2024252600000000EA
:10936000000064040100040000000000000C001074
:1093700028303400F470FF7F01000000000000007E
:10938000CC1000000000000000001A0000000000E7
:10939000FF00000000000000088A000883040000AD
:1093A000138A000850040000218A00080100000010
:1093B0000000000000960000000008009600000079
:1093C0000008000004000000709200080000000087
:1093D000000000000000000000000000000000008D
:0493E0000000000089
:00000001FF
